:020000041100E9
:10300000002373B52B4D2C4C28006361022601F080
:103010006DF94021FE2221742800284B009601F012
:10302000B7F9002836D1217CFF222800244B0096D6
:1030300001F0AEF900282DD1224BA2899A4226D167
:10304000E389214A93420DD1204B6361204B2268D2
:10305000002A03D1002B01D043CB43C4280001F048
:1030600083F973BD1B4A934201D00023EFE71A4B4B
:103070001A4A1B68934206D9C02304222800217CE7
:103080009B0001F0FBF9114B6361154BDFE7002357
:103090002374EAE7CC233821AC2228009B01217459
:1030A00001F0ECF90028F2D10E4B63610E4BE38185
:1030B0000E4BCCE7643CFF1FFC5BFF1F085CFF1F4F
:1030C0000A5CFF1F595900008305000019410011D7
:1030D000F0B8001182150000205CFF1F871300006C
:1030E000FCB80011D1410011AAAAFFFFE4B80011F9
:1030F000F7B5164B0192C318021D002000938823D8
:103100005B05D3181B685C1C1AD09CB2402C18D8E5
:103110008D781E0CAC466746CD782D023D43AE42FD
:1031200006D1019800280ED110000C70240A4C70B2
:1031300003249BB20733A343D218009B9A42DED3E9
:10314000FEBD4432F9E71000FAE7C046FC0F00006C
:10315000802213B503000324019189B25201073183
:103160009B18A14304305A1A88235B05C3181B68B7
:10317000591C03D190429241104016BD99B240298A
:1031800007D80B000733A343C0189042ECD30020AC
:10319000F3E74430F9E7134B134A1B68126810B584
:1031A000FA24934201D81A00F824104BE4021B6859
:1031B0009A4210D813000E4A12689A420ED3013375
:1031C00007D1F823DB029C4203D10A49054808F0E5
:1031D000EBFA200010BDFC24E402ECE7FE24E4023C
:1031E000F7E7C04600C0071100D0071100E0071143
:1031F00000F00711FFFFFF7FF0B59BB015000490B2
:103200000391402A00D9A0E006AB59801A80FFF74D
:10321000C2FF0400042816D9002206A9FFF768FFA0
:10322000052810D906AB1B88AB420CD1002D07D066
:10323000514B2A000499C01808F07EF9002802D1E9
:1032400001201BB0F0BD06AB1D8020000699FFF7E2
:103250007FFF041E7BD1069B0793FFF79CFF802313
:103260005B01C618802307001B039E4201D3F8268A
:10327000F60288235B05F31801931B68013302D023
:10328000019808F0B1F83D49019808F08DFA3B1D0E
:103290000293331D05938822029B52059B181B68DD
:1032A00008935A1C3CD044219AB20091402A04D879
:1032B0000320D11D814389B2009103991B0C8B42DD
:1032C00024D0402A22D80122300008A9FFF710FF9D
:1032D000021E1BD1380008A9FFF70AFF04000428CA
:1032E00031D9009A059B9B1880225201B218934253
:1032F00040D288235B05C118009A09A808F03CFA5F
:103300001D4B009A09A9F01808F09EF8009A029B3C
:103310009446634402931A4B029AFB189A42BAD31A
:1033200088235B05FC1821680198013908F03CFAF4
:10333000200008F059F8039A07AB5A80300007992B
:10334000FFF706FF0400002C03D1002079E70428D2
:10335000FBD988235B05E018069908F025FA0323BA
:10336000EA1C9A4300D16BE7034B0499E01808F07C
:103370006BF865E70424ECE704000011FFFFFF7F12
:10338000F80F0000F7B505001400402A21D80027E7
:1033900001AE71803780FFF7FEFE042816D93A008F
:1033A0003100FFF7A5FE042810D93688BC420BD0A7
:1033B000BD4209D0221CB44200D9321C064B92B245
:1033C000C118280008F0D8F930B2FEBDC04300B2E1
:1033D000FBE703204042F8E70400001137B5042260
:1033E00004000D0001A81649FFF7CCFF02000428D5
:1033F0000BD1019BA34208D3AB4204D0104901A8D2
:103400000195FFF7F9FE01203EBD0E4C2368200018
:10341000019307F0E9FF019920000139019108F0BB
:10342000C3F980235B01E418074B9C42EED10422D0
:10343000034901A80195FFF7DFFE0020E4E7C0463D
:103440005555000000C007110000081130B589B0C3
:1034500008F0F2F810226946254807F0FDFE254BDA
:10346000009A9A420ED1019B029A0F2B33D8002169
:1034700001240698013B08D2002900D00292029B49
:10348000013331D10023029325E0551CF2D1020013
:103490002100EFE710341022200004A907F0DCFE21
:1034A000029B013301D1069B0293882304995B059B
:1034B000C918059B06981A03120B049105928142C4
:1034C00003D02B4201D108F057F9019B013B019336
:1034D000019B002BDED1029B002B03D004930498A8
:1034E0004168084709B030BDE025014C2D03EFE7E6
:1034F00000000111504859368022F8B5964C974B80
:10350000D200002120001C6007F00EFF2300944A27
:1035100088331A60934B1A786A23002A00D011333B
:10352000E3620A232365904B37221B780821A363AB
:103530008E4B6018E361102323628D4B3B25636142
:10354000C823DB00A36123008C331A602823013ACF
:10355000E26321646364C267043A201DC2672000ED
:10356000BC3005602000C03001602000C430036022
:1035700020000635CC3005602000083DC8300560CD
:103580002000D03002602200D43211602200D832F4
:10359000136022000226E032200016604222DC3056
:1035A000026020001B3DE43005602000E83001602F
:1035B0002000EC30036023000520F4331860230062
:1035C000F0331A602300183290331A6023009433CA
:1035D000196023001E3A98331A60AF23DB00236082
:1035E000644BFA252363644B6448A3642300B93217
:1035F000FC33FF32AD00A260E56022611D60A06275
:103600007320E0656D386065A065FA2796203F015C
:103610008000E76465625960A0660920E0660020CA
:10362000616757496666E167564E57492667A06746
:103630000F601527676027001A219C373960270023
:103640000731A037396027004B49A837396021007E
:10365000F8310D6021006427A4310F6021005F3F25
:10366000AC310F602100033FB0310F602700B43749
:103670003D00C8272F6027003825B83738609D6087
:10368000424D96215D64424D8900DD61414D1962D4
:103690005D62F53DFF3D9D621E253949DD66596637
:1036A000996499673C49DE651E6618675867D96753
:1036B000BE233A495B00E1508130394BFF30235043
:1036C00004302150C42149006350C623E4205B002C
:1036D000E2500433E2503349334A344BD160344929
:1036E000800019503349E938FF3819503249043005
:1036F000195032493248D16132491163324951631C
:103700001900F4310860CE20304940001160304982
:10371000195019002F48F83108602F49D1658221CE
:103720002E4A89005A501A002D490832D1671A00D2
:103730002C49B432116088212B4A89005A501A0052
:103740002A49883211602A4ADA6407F045FD0120CF
:1037500007F082FFF8BDC0460004FF1F985EFF1F00
:103760007069FF1F903EFF1F4A0AFF1F3A070000C3
:1037700080C3C9019A02000050C300006A1800000B
:1037800088130000204E0000F009FF1F6509FF1F8D
:1037900068100000C4090000DC05000040420F0072
:1037A00010270000D91AFF1FFC00FF1F0000FF1F99
:1037B0008127FF1FC52AFF1F5D29FF1F251EFF1F31
:1037C0007523FF1F411EFF1FED1FFF1FB11DFF1FB0
:1037D0000124FF1FE924FF1FD918FF1FB923FF1F72
:1037E000C921FF1FD521FF1FB11CFF1F691DFF1F2E
:1037F0009D1CFF1F0223F0B50124604D604E2B700D
:10380000604B91B01C70604F039333680021082017
:10381000BB7006F0F3FB082006F0EAFA002398429A
:1038200005D0BA78552A02D0332A00D09AE0336006
:1038300007F0BAFEFFF760FE1F2201240021534B60
:1038400010AE1A70524B1C70524B1970524B1968C3
:103850009143163A0A431A60602219689143403A2C
:103860000A431A6007F0F0FC07F0B6FEC120FF2102
:103870004A4B80001A588A431A50C5229200985821
:103880008843BF39014399509858454908408021E1
:10389000C9010143802099509958C0050902090ABD
:1038A0000143995080213F48490107F0ADFE0323B1
:1038B00022003D49019400933C4807F00DFD2C2265
:1038C0003B4905A807F058FF05AC61782078023421
:1038D00006F0AEFAA642F8D1364C0121002006F0DF
:1038E000BBFB0920012106F0B7FB2268324B032005
:1038F0001A40A023DB0213432360802322689B0429
:103900001343236022682D4B1A4080239B031343EB
:1039100023602B4A2B4B934200D8012007F0FCFC7C
:1039200007F062FE80232268DB04134323602878BB
:1039300007F0DAFD039B1878C0B207F0EDFE07F040
:10394000ABFC2149042007F027FE06F09DFC00F0A7
:10395000A7F800F0BFFD00F067FE00F00BFA0020B2
:1039600011B0F0BD00932100174A042007F07CFE3F
:103970008023DB059C62FFF769FD59E74A0AFF1FB8
:1039800034F00040903EFF1F2C5CFF1F480AFF1FD1
:10399000490AFF1F680AFF1FBCF0004000E100E079
:1039A000FF00FFFF943EFF1F1851FF1F944EFF1FA3
:1039B00008B8001114F00040FF7FF8FFFFFF9FFFE1
:1039C0000080FF1F7069FF1F3B00010870B50025D4
:1039D0002549264A26484D6308CA1B051B0DED18CC
:1039E0008242F9D100268022224B92058B63092165
:1039F000214B224C1E62224B1120DA67214BDA68E0
:103A00008A43DA609A6820490A409A60266007F083
:103A1000D3FC112007F050FD8022636C9343636454
:103A2000EE24E4006C43194A200C04006423904205
:103A30000AD8FA223300D200904205D9144B0A2149
:103A4000C01807F009FDC3B2124A11201372D480C6
:103A500007F04AFC104B1B78002B04D10F4B1021B0
:103A6000187807F009FD70BD000005408805054085
:103A700000060540FF01000000F000400038004053
:103A800004E100E03CF00040FFDFFFFFB70B000067
:103A900030F8FFFF145CFF1F4E5EFF1F4C5CFF1FE2
:103AA000002210B51100112007F0EEFB10BD000040
:103AB000F8B500230926374F374C3B62E3681120E5
:103AC000B343E36007F0F8FC112007F075FC112008
:103AD00007F0F2FB402322688025134323608023F4
:103AE0006268DB0213436360A3682C4A2B43A36024
:103AF000A36802211340A3608023A2689B011343A3
:103B00001022A360236C072093432364236C0F3A95
:103B10001343236480235B003B62226B204B1A40DB
:103B20002263626B1A406263A26B1A40A263E26B6B
:103B30001340E363E3681B4A1340E36006F078F93F
:103B40000121072006F088FA174B11205A6C154303
:103B50005D6407F0F1FDFD21144B154A89005A50B0
:103B60008023C720626B5B0313436363E3688000B9
:103B70003343E3600F4B104A195811408022120260
:103B80000A431A50802292051A6008220B4B5A638E
:103B9000F8BDC04600F000403CF00040FFFFDFFFF2
:103BA000EFFFEFFFFFFF7FFF003800400000FF1F27
:103BB000CD39001100E100E0FF00FFFF00000540EB
:103BC00030B503A804880B20002C0ED14968074D9E
:103BD00008784978090201430A20A94205D1012148
:103BE00020001980024B1B7A137030BD192A000087
:103BF000145CFF1FF7B5150008AA16884A680F4F16
:103C000014785278120222430A24BA4214D10122B3
:103C1000DBB2019200962A0007F070FA041E0BD165
:103C2000074B1B68002B07D068782A7800021043E6
:103C300042425041013098472000FEBD0229000059
:103C4000985BFF1F30B5012503790400BFB02B42FC
:103C500011D00A49408806F0BDFD28420BD0084B20
:103C600001A95B8D4D800B80064B00221B7A60887A
:103C70000B7103F0A5FE3FB030BDC046905BFF1F47
:103C8000D83AFF1F145CFF1F10B50549054806F020
:103C900057FD0421044A054806F014FD10BDC04636
:103CA000905BFF1FFFFF000034B80011D83AFF1FE0
:103CB00010B5024804F006FD10BDC046453C001199
:103CC000062310B5837010330371443B43712A33CC
:103CD00083714433C37100230222012103720E4B0E
:103CE000027041701C8881724472197A0273C17229
:103CF0009A784273DA7882730322C2731A79027453
:103D00005A7942740C2282749A79C274DB790375F1
:103D10001123C370152010BD145CFF1F10B51420B3
:103D200007F092FC124B14220021186007F0FCFAF5
:103D3000002007F001FB012007F056FA022007F0EF
:103D40006BFC032003F062FF042005F077FF0520E1
:103D500003F0A0F9062003F06DFE072001F004FA3D
:103D6000082006F08FFC092000F0E6FF10BDC046D9
:103D70009C5BFF1F07F010FB012007F0FDFB07F025
:103D8000C3FC0000094B10B50400984205D001297E
:103D900004D12000064906F0D3FC10BD0229FCD155
:103DA000013904F04DFC0028F3D0F6E7FEFF0000D7
:103DB000C25BFF1F70B50D7A100004AA2C00168894
:103DC00010221440154220D1002E20D10A78022A58
:103DD00018D14A68517815780E4A09022943914250
:103DE00005D00D4A914209D01C800A2404E0142217
:103DF0000A491A8007F0C0FC200070BD0C22084957
:103E00001A80F7E71C800124F6E70824F4E70B2466
:103E1000F2E7C046F3FF0000F4FF0000203DFF1F63
:103E200014B9001110B504000749084806F088FCD1
:103E3000074804F087FB0020E40704D50721054A62
:103E4000054806F03FFC10BDC25BFF1FFFFF0000EE
:103E5000853D001178B800111C3BFF1F00B50C4BCD
:103E6000BFB01A780B4902A800F098FC6B4680B2EC
:103E7000D880002809D06A46074B01A91B88938087
:103E8000064B0022188803F09BFD3FB000BDC046E2
:103E9000A05BFF1FA15BFF1F763BFF1F803CFF1F46
:103EA00000B50C4BBFB01A780B4902A801F0CEFC4C
:103EB0006B4680B2D880002809D06A46074B01A91A
:103EC0005B8D9380064B0022188803F079FD3FB08C
:103ED00000BDC046CA5BFF1FCB5BFF1F1C3BFF1F23
:103EE000803CFF1FF7B50E00377A1C0008AB1100AD
:103EF0003D001A8820231D401F423CD13378022BFD
:103F00003BD173681F785B781B023B431E4FBB425B
:103F100008D01E4FBB4214D01D4DAB4221D00A2504
:103F20002800FEBD002A2AD1142C2AD82200F068CD
:103F300007F022FC174B1C70012CF1D9FFF7B0FFE2
:103F4000EEE7002A1BD1202C1BD82200F06807F0D6
:103F500013FC114B04211C70104B187807F08CFADD
:103F6000DEE7E3B20124009201940A00310007F079
:103F7000C5F80500D4E70825D2E70125D0E70B25D1
:103F8000CEE70D25CCE7C046F3FF0000F4FF0000AC
:103F900002290000CA5BFF1FA05BFF1F4C5CFF1FD4
:103FA000332310B5040003700A220749013007F0DB
:103FB000E3FB064B0F201B681A0AE37222731A0CEC
:103FC0001B0E6273A37310BD145CFF1F3C5CFF1FCC
:103FD00030B5012503790400BFB02B4213D00B4943
:103FE000408806F0F7FB28420DD06A46084B02A82D
:103FF0001B889380FFF7D4FF6B46D880002260882F
:1040000001A903F0DDFC3FB030BDC046C25BFF1F1D
:10401000763BFF1F10B5024804F054FB10BDC046AC
:10402000D13F001170B5160004AA148805AA1578AE
:104030004A685078117800022A4A084380180528F7
:104040004BD807F029FA03131E29343F0720042C0C
:104050000BD80522121BAA4200D92A0022491A8035
:104060003000091907F088FB002070BD0720112CD3
:10407000FBD81222121BAA4200D92A001B491A801F
:10408000EEE707200E2CF0D80F22121BAA4200D90F
:104090002A0017491A80E3E70720032CE5D80422F9
:1040A000121BAA4200D92A0012491A80D8E7072019
:1040B000032CDAD80422121BAA4200D92A000E4986
:1040C0001A80CDE70720032CCFD80422121BAA4266
:1040D00000D92A0009491A80C2E700220A201A8062
:1040E000C3E7C046DCD5FFFFC3B80011E85BFF1F84
:1040F000B3B80011AEB80011A9B80011A4B80011EE
:1041000010B50D21024A034806F0DCFA10BDC04686
:1041100098B800118C3BFF1FF0B50024274E85B0E6
:104120003000B47100F0E2F8254D264BEA89297C75
:104130009A422FD10423300003AA00F057F904005B
:10414000300000F011F90123B371002C34D16B461B
:1041500099892B68C9BA4B4329891B4A1B145B18E0
:1041600053806B46D9896B6849BA89B24B436989D8
:104170001B0C5B181548191C1BB2834200DD011C87
:104180000B0400D500211388918001331380200097
:1041900005B0F0BD0227220003AB3000009700F00D
:1041A000F7F80E230400297C0122300000976B44AD
:1041B00000F0EEF80443C3E71C00E8E7643CFF1F8F
:1041C000FC5BFF1F83050000145CFF1F0F2700002E
:1041D00073B5234E300000F089F8224D07236A465C
:1041E0003000297C00F002F904003000002C33D1AB
:1041F0006B461B787F2B2FD800F0B6F86B46D8782B
:10420000F02302041B031A406B469B8816495BBAD5
:104210009BB21A432B68000953432A891B0C9B1835
:104220004B806B465A789B7812031B011A436B68CC
:10423000024353436A891B0C9B180C481A1C1BB27F
:10424000834200DD021C130400D500220B888A8003
:1042500001330B80200076BD00F086F80124F9E7D9
:10426000643CFF1FFC5BFF1F145CFF1F0F27000057
:1042700070B5114C237C002B0FD0382B0ED10F4D75
:10428000280000F033F8CC23AC222800217C9B01CD
:1042900000F0F4F8280000F067F870BD084BE289E0
:1042A0009A42FAD1054D280000F020F8002228009B
:1042B000217C00F0C5F8EDE7FC5BFF1F643CFF1FAD
:1042C0008305000010B5084B1A7C002A09D05B69F1
:1042D000002B06D09847041E01D0FEF791FE200067
:1042E00010BD0124F9E7C046FC5BFF1F70B5C17922
:1042F00005000C00631E9C411A4BE402E4184900BF
:104300000460C9B2007905F0DDFEE97968794900F9
:104310000131C9B205F0D6FEE8790930C0B206F025
:10432000CBFF0023E36661332360AA795B3B002A5D
:104330000ED022689A43023B134323600A23E361B1
:104340000733236200232363A3630133E36370BD58
:1043500022689A4302231343236046236361063392
:10436000A361EFE70050004070B50025040003682A
:10437000DD66C0790930C0B207F09EF829002079C7
:1043800005F03CFE2900607905F038FE70BD0000A4
:10439000F8B51E0006AB1D78002304681700E3661D
:1043A000616007F049F901238022E3662B00276151
:1043B0005200013B08D206F02FFF08200A4A11687C
:1043C000002D03D12800F8BD2261F2E7236F0342DC
:1043D00003D02369013D3370013613685B1A032B48
:1043E000EED90125EEE7C0466008FF1F70B51C003E
:1043F000002305681600EB66696007F01DF90123CC
:104400008022EB6623005200013B08D206F004FF35
:1044100008200A4A1168002C03D1200070BD2A61CF
:10442000F2E72B6F034203D02B69013C3370013656
:1044300013685B1A032BEED90124EEE76008FF1F17
:10444000002370B504681500E366616007F0F4F8B6
:104450000123E366256106F0DFFE8020064A800026
:104460001168636B034205D113685B1A032BF8D9FB
:10447000012070BD0020FCE76008FF1F70B51D0023
:10448000002304681600E366616007F0D5F8012395
:10449000E36626610F33626B1A42FCD02B0A23615C
:1044A0001023626B1A42FCD0EDB2256106F0B4FE17
:1044B0008020074A80001168636B034205D11368AE
:1044C0005B1A032BF8D9012070BD0020FCE7C04621
:1044D0006008FF1F10B5084CE368002B08D180224C
:1044E000064B52021B689B186360054B1B682360D8
:1044F00007F06AF8A06010BD3C5CFF1FC8F00040E8
:10450000CCF0004070B5184A936A916A9942FBD189
:1045100016498A689A421FD39A1A8B60144B012657
:10452000186893B2D202D20E4343424300204C6833
:104530001B0A1B1912029B180E4C0A684B60551C73
:10454000A3420CD8002801D04B600A600A4A1360CD
:1045500008680A4B186070BD581E821ADDE7084AC9
:1045600030009B182A00EAE700F000403C5CFF1F87
:10457000140AFF1F40420F00C8F00040CCF000407A
:10458000C0BDF0FF70B51F4C23793F2B01D93F23ED
:1045900023711D4B22791A701878C0B207F09CF86D
:1045A00018231A491A4A0B801A4913800B8053802A
:1045B000A379194980200B800C21938001334B4350
:1045C000164D191C0001834200D9011C2980D1809D
:1045D0006379002B11D101336371237A012B01D848
:1045E000022323726279237A0D4853430A215843E8
:1045F00006F032FF0B4D286070BDA02BEDD9A02333
:10460000EAE7C046305CFF1F480AFF1F7E3CFF1FE1
:104610003C3EFF1F7C3CFF1F7A3CFF1F783CFF1F86
:1046200071020000205CFF1FF8B514210020FEF786
:10463000D5FE114C011E114D09D10C22104BC1CBDE
:10464000C1C4280006F070FEFFF79CFFF8BD0C22E5
:1046500020000C49FEF796FE0C2802D0084B43CBF5
:1046600043C40C2228000849FEF78CFE0C28EBD02E
:104670000C220021E5E7C046305CFF1FFC5BFF1FFA
:1046800008B90011FC0C0000F50C0000F0B51D4C41
:104690008022A5440400882069465201400506F0A6
:1046A00093FD902212016A441300200032C832C3E5
:1046B00016C816C38023144C144FA6689B033343BB
:1046C000A3603B6006F078FF8823A0685B05C018F4
:1046D00006F08AFE0025882329008022A0685B0559
:1046E000C01840196944520006F0AEFE802301351F
:1046F000FF355B019D42EED1A6603E60044B9D44B8
:10470000F0BDC046FCEFFFFFB03DFF1F9808FF1F44
:1047100004100000F0B5040087B0002825D06846DA
:1047200006F0D2FD1B4C022806D106226946200065
:1047300006F002FF002816D06946002301250F2647
:104740002F00E25C013310091030874038002F0041
:10475000324097403A0002434A610439062BEFD1B8
:104760006846FFF793FF07B0F0BD182269460A4874
:1047700006F02AFD6A46A300D358013305D018225B
:10478000FF21684606F0D0FDEAE70134062CF1D19E
:10479000E9E7C0466509FF1F00090011F0B50025D3
:1047A00004000E0085B0AA4200D183E04B1C0878BB
:1047B00001934B788978377909021943F3783F06DA
:1047C0001B040B431F43039720706570252800D1FD
:1047D00093E033D8112813D806F0C6FE66000D0109
:1047E0000D010D010D01A700B500AE000D010D0179
:1047F0000D010D010D010D010D010D01E700070176
:10480000232800D1C0E0DB2800D016E1042A00D81C
:10481000A9E01025052A05D0551F2A003800711D72
:1048200006F0AAFF05223100200006F0A5FF2A00AD
:104830003900601D06F0A0FF05353BE0562856D034
:1048400010D8332800D19AE0552836D02628DAD15E
:10485000894B2900132218001D0006F065FDFEF7A4
:10486000CFFB59E0712800D174E0722800D17DE0BF
:10487000DC28C8D1022A00D875E07378BFB2637013
:10488000B378A370032A05D0033A390092B2F01C22
:10489000FEF7B2FC10223900E01CFEF773FDC51CC8
:1048A000002807DA60705CE00C222000734906F0F3
:1048B00063FF0C25280005B0F0BD013A704D0C2AAD
:1048C00013D8002A0AD02800019906F055FFFFF7F7
:1048D00059FE0C2228006B49FEF78EFC29000C22A1
:1048E000601C06F049FF0D25E4E70C22EBE7644D60
:1048F000654B2A0043CB43C2E9E7013A5E4D0C2ADF
:1049000011D8002A08D00199280006F035FF0C22A2
:1049100028005E49FEF770FC29001322601C06F097
:104920002BFF1425C6E70C22EDE705225849601C31
:1049300006F022FF0625BDE712225649601C06F04C
:104940001BFF1325B6E708225349601C06F014FF2D
:104950000925AFE77178F02905D8504B188801F088
:10496000D1FB0225A6E7FF236370FAE74C4B012A2F
:1049700003D072785A706270F3E75B78F4E7200036
:10498000FFF70EFB050095E7042A04D9454D2F607B
:1049900006F01AFEA860FFF7B5FD0422039003A9F4
:1049A000601C06F0E9FE052584E73F4D062A15D96F
:1049B00006222800019906F0BFFD00280ED006222D
:1049C0000199280006F0D8FE062238492800FEF793
:1049D00013FC0123324A51780B43537029000622FD
:1049E000601C06F0C9FE072564E7012ABBD0707879
:1049F000FFF790FEB5E7012800D004E7931E2C4F87
:104A00001A2B04D87378002B09D100F009F9294B2F
:104A100039001D78601C6A1E06F0AEFE4AE7551E7E
:104A20002A000199380006F0A7FE2349AAB23800EF
:104A3000FEF7E2FB00F02AF9E9E7DA2893D1042A2D
:104A400091D9082A15D9B37972791B021343F279E7
:104A500012041A43337A1B0613433B603B6805225A
:104A600031002000039306F087FE0422601D03A995
:104A70006CE7FE236370F1E7FC5BFF1F14B90011C4
:104A8000305CFF1FFC0C000008B90011F50C0000A1
:104A9000085CFF1FE85BFF1FB43DFF1F803CFF1F4A
:104AA0002C5CFF1F3C5CFF1F6509FF1FADAC0000C5
:104AB0002D5EFF1F2B5EFF1FAEDE00007047000063
:104AC000020010B5094B0A32094C92B2DA815A82BF
:104AD00098811882207802F07BF90422054B01218D
:104AE00020781A7006F0C8FC10BDC0463E3DFF1F7E
:104AF000765EFF1F755EFF1F013870B5042809D868
:104B000006F0CAFC0309230812001E4B0221187884
:104B100006F0B2FC70BD1B4B0821187806F054FE5D
:104B20000022194B1A72F5E780220024164B154D0E
:104B300052001A81082128781A68DC7206F07CFC81
:104B40002100287806F0E8FCE4E70E4B08211878ED
:104B500006F03AFE0D48FFF7B3F80D4B0D4A9B796E
:104B600093800D4A13800022074BDA720132FF3224
:104B70001A810A4B5B78002BCCD0094A136006F0EF
:104B80000BFEC7E74C5CFF1F205CFF1F893CFF1F2B
:104B9000305CFF1F3C3EFF1F7A3CFF1F2C5CFF1F59
:104BA00034F0004010B5002905D1082803D10131A7
:104BB000013005F051FA10BD10B501290FD10828B8
:104BC0000DD10021013005F047FA054B1B78002B71
:104BD00005D02622034B04485A72FFF771FF10BD1F
:104BE0004E5EFF1F205CFF1FC40900000300F0B5EC
:104BF0000A4D8E18B14202D152008018F0BD0C78D7
:104C00002F6824093C5D0F271C700C7801313C4053
:104C10002F683C5D5C700233ECE7C046743CFF1FBC
:104C20000E22114B10B51A700D23104C1049237031
:104C3000093A043B0F48637006F09EFD2D230122C4
:104C40000D490E48E371FFF7D1FF01220C49FFF730
:104C5000CDFF01220B49FFF7C9FF00220A491000CE
:104C6000FEF7CAFA10BDC0464A5EFF1F2B5EFF1F4B
:104C7000C3B800112D5EFF1F6709FF1F335EFF1FC2
:104C80006609FF1F6509FF1FAEDE000070B5124CFC
:104C9000132220001149FEF775FB114D002817DD86
:104CA000AB78002B14D0431C2B7009236B700023AE
:104CB00000190370287829000130C0B206F0E4FB27
:104CC000297822000139C9B2002005F019FC70BD15
:104CD000FFF7A6FFEEE7C0462D5EFF1FAEDE000029
:104CE0002B5EFF1F10B5114B1A781870002A0ED0DA
:104CF00000280BD10E4B1A78062A07D85423D3402C
:104D0000DB0703D50B4B187802F062F810BD0028C2
:104D1000FCD0074B1B78012B02D0033B022BF5D8AC
:104D2000044B0121187806F0A7FBEFE74E5EFF1F4A
:104D3000755EFF1F765EFF1F70B5504E504A514999
:104D40003070082005F07EFA0121092005F084F971
:104D5000092005F065FA0121002005F07DF9002009
:104D600005F05EFAFEF74CF906F0EEFB0322464929
:104D70004648FFF73BFF2D24030004221C704449E2
:104D80000130FFF733FF30230470424D424C437033
:104D900083702E3B062220004049EB87FEF7F2FA93
:104DA000062813D0200006F08FFA022809D003212C
:104DB000200006F0A1FC8D23E3706E3B23711933B4
:104DC0006371062220003549FEF716FA344B1B6842
:104DD000FC335C64FFF75AFF0020FFF783FF314C80
:104DE000314A0121314B1278207801F0B3FF304A6B
:104DF000304B12780021207801F0ACFF01222E4BBD
:104E00001A702E4B9B78552B31D12D4B3B325A7259
:104E10002C4B2D4AAB81EA812B826A82202130788B
:104E200006F0A2FA0120404205F0B6FB0120404204
:104E300005F052FCFFF764F9FEF726FF00F09EFC38
:104E400001204042FEF7EEFF012006F07DFAF0203F
:104E500001F03CF90121307806F00EFB307802F0C9
:104E600013F91A4806F060FCFEF722FE70BD6422BA
:104E7000174B5B7953431A000A32CBE74C5CFF1F98
:104E8000A54B0011B94B0011B43DFF1FE85BFF1F9C
:104E9000085CFF1F3E3DFF1F6509FF1FADAC000012
:104EA000985EFF1F765EFF1FA83CFF1F893CFF1F17
:104EB0004A5EFF1F2B5EFF1F1C5EFF1F2C5CFF1F47
:104EC000205CFF1FC4090000CE0900004E5CFF1FDC
:104ED000305CFF1FF8B50A0020230D001A4019426C
:104EE00051D0544B1B78002B3CD0FFF70BFB524B9F
:104EF000524C534E99686268737A8A1ADB039A425D
:104F000002D36160FEF7D4FD327A217A531EDBB200
:104F100099422AD1FFF7ACF9637A002B1FD0013BED
:104F2000DBB26372002B1AD1464B9B78552B01D113
:104F300006F032FCE37A002B0CD00023424A434FA8
:104F4000E3721388380001331380FEF7B9FE39008D
:104F500006F08AF9642370795843FFF7B1FD237A8C
:104F60000133237220206840F8BD9142D4D300233E
:104F70002372FFF7A7F9354F3800FEF7A1FE39007D
:104F800006F072F9C8E70BB2002B0ADA304B18783A
:104F900006F04AFB002801D006F0A6FB80200002A4
:104FA000E1E70224214206D0244B01201A72FFF7C8
:104FB00099FE2000D7E70B071BD5FFF7A3FA1E4B7E
:104FC0001E491F4C98684A68637A821ADB039A422A
:104FD00002D34860FEF76CFDFFF774F9FFF748F95C
:104FE00000F0E6FB2368DB0701D5FFF713F8082084
:104FF000B9E710240E002640214206D00D4B1B7845
:10500000002BD6D1FEF754FED3E70124214209D06C
:10501000104800F06DF806F0E7FB3100092005F0BC
:105020001BF8C6E704240800204021429CD0FEF76C
:1050300015FFBEE74E5EFF1F3C5CFF1F205CFF1F9D
:10504000305CFF1F2C5CFF1F145CFF1F893CFF1F9F
:105050004C5CFF1F6C3CFF1FF0B51B4B1B4F1B88AC
:105060003A8804001A4E1B4D85B09A420DD83288FA
:105070009A420AD3184B1A882B889A4205D1174AAC
:10508000174B12881B889A421BD0052001F074F838
:105090003B8802AA13803388019053802B88114DDE
:1050A00093800F4B02A91B88D3800F4B2A78188856
:1050B00002F090FD0D4B08212878019A1C7006F033
:1050C000A3F805B0F0BDC0461A5EFF1F7E3CFF1F6F
:1050D0007C3CFF1F7A3CFF1F185EFF1F165EFF1F00
:1050E000783CFF1F765EFF1F803CFF1F145EFF1F92
:1050F00013B50C4B1C78002C11D1002801D00A4BA1
:1051000018600A4A0A4B11780A4A10780A4A019232
:105110000A4A0092002205F0EBF8200016BD112487
:10512000FBE7C046755EFF1F105EFF1F745EFF1F2A
:10513000645EFF1F765EFF1F505EFF1F545EFF1F01
:1051400010B5064B12201B78052B06D1044B1322F9
:105150001988044B187801F0EBF910BD755EFF1F3C
:10516000803CFF1F765EFF1F10B500240122114B0B
:1051700052421870104B1C70104B1A8001F084FFC3
:1051800004220F4B21001A700E480C3206F04CF826
:10519000102221000C4806F047F807220B4B1C6038
:1051A0000B4B1C700B4B1C700B4B1A700B4B1C7079
:1051B00010BDC046765EFF1F755EFF1F803CFF1F5F
:1051C000745EFF1F645EFF1F545EFF1F505EFF1F73
:1051D0002A5EFF1F295EFF1F823CFF1F285EFF1F04
:1051E000F8B5174C0600257806A814240078052D7C
:1051F00023D1B41F134FA5B21824BD421DD88D1F53
:10520000ADB2BD4219D8FA256D00AA4215D21D00D3
:105210000D4F0A3DADB2BD420FD80C4C26800C4C50
:1052200021800C4900240A800B4A1380FFF714FFE9
:105230000A4B0421187806F0C7FA2000F8BDC046D2
:10524000755EFF1F790C0000750C00007E3CFF1F8F
:105250007C3CFF1F7A3CFF1F783CFF1F765EFF1FE0
:10526000F0B50BB20D0089B0002B00DB70E1A44E4D
:10527000307806F0D9F9041E50D00378A22B00D163
:1052800022E1D02B1AD0912B45D143780E2B42D15D
:105290009C4B82889A423ED19B4A83681278052AA9
:1052A00039D1032018567F2835D0984B1B68002B26
:1052B00031D05B68002B2ED098472CE080780728EF
:1052C00029D806F0E9F80428183F3F74A8D8637875
:1052D000002B0CD101218C4B19708D4B1A78002AB0
:1052E0005BD08C4B307801F035FD002855D007227B
:1052F000854B1A7051E061780029F8D1E378002BD2
:1053000011D0854A854B1278307801F023FD60700A
:105310006378002BEBD1200006F0E6F98020000234
:10532000684009B0F0BD784B1B78022BF3D0012107
:10533000307806F041FA0028EAD10121307806F0F1
:105340009BF8E5E76378002BD1D16F4F032807D195
:105350003B78052B02D101333B701EE00223FBE7B3
:105360006F4B1A886F4B0293002A0BD01B78002BCF
:1053700003D00121307805F047FF3B78062B04D19C
:10538000013BE9E7029B1A70F7E7042B41D10121A9
:10539000029B3078197006F06FF85C4B1B68002B8D
:1053A000B9D01B68002BB6D0574A107884E76378D1
:1053B000554F002B27D10622211D5B4806F0DCF952
:1053C00062895A4B5A491A80A2895A4B1A80E3893A
:1053D0000B800521397058490A80584A1380228A67
:1053E000574B1A80574B1B78012B09D11F2000F017
:1053F000C3FEFA22920042430421307805F004FFF4
:105400000022484B75E7312B00D070E70022454B56
:105410001A700323A0E706220021434805F004FF89
:105420000023454A04211380444A30781380444ABB
:10543000138006F0C9F90821307806F0C5F9A37980
:10544000083B5A425341304A03331370304B1B78A8
:10545000002B06D0334B30781A78002A06D001F0A2
:10546000B7FC0122314B52421A8096E70121197094
:1054700006F002F8F5E70821307806F0A5F9637820
:10548000002B00D047E72C4B2D4F0293E388029A64
:1054900004211380294B307803932389039A1380C6
:1054A00063893B8006F088F9002800D033E7264B5B
:1054B0001B68002B00D12EE7039902983A880988CF
:1054C00000881B68984726E74379132B00D022E712
:1054D0000389012B0AD11D4B1B78022B06D1082111
:1054E000307806F071F9FFF72BFE14E7052000F085
:1054F00043FE08210200307805F086FE0BE7C04627
:10550000765EFF1F05140000755EFF1F105EFF1F13
:10551000A83CFF1F893CFF1F4A5EFF1F2B5EFF1F39
:105520004C5EFF1F4E5EFF1F1D5EFF1F803CFF1F76
:10553000245EFF1F265EFF1F1A5EFF1F185EFF1FFF
:10554000165EFF1F1C5EFF1F0C5EFF1F145EFF1F19
:105550008020C001014200D0E2E6CB0731D5324BBA
:105560001B78002B1DD0314E05AC3378052B1AD19A
:10557000023B23702E4B21001B7823722D4B1B788E
:1055800063722D4B187801F089FB002809D00720A1
:105590002A4B30701B68002B03D01B68002B00D0F7
:1055A00098470120BCE60E20254B06221B78254992
:1055B0002370254B1B78637002ABC01806F0DCF833
:1055C000D8E7022308001840194209D0174B1B786E
:1055D000052B03D11D4B188805F02EFE02209FE6F7
:1055E0000424214203D0FFF737FD200098E608236A
:1055F00008001840194200D193E6154B1C78012C85
:1056000003D0022C0DD008208AE6124B124A13490F
:1056100013481B881288098800880094FFF7E0FD72
:10562000F1E7FFF78DFDEEE74E5EFF1F755EFF1F92
:10563000823CFF1F285EFF1F765EFF1F105EFF1F6C
:105640002A5EFF1F833CFF1F295EFF1F803CFF1F58
:10565000145EFF1F783CFF1F7A3CFF1F7C3CFF1F3E
:105660007E3CFF1F10B502A804880B20002C10D12F
:10567000496808784978090201430C48814209D1F8
:10568000022119800A4B59881170DB7800205BB227
:10569000537010BD074C0A20A142FAD10221198093
:1056A000034B998811705B79F0E7C0466E2A0000C1
:1056B000145CFF1F6F2A0000F7B5150008AA1688B2
:1056C0004A680F4F14785278120222430A24BA42D1
:1056D00014D10122DBB2019200962A0005F00EFDE2
:1056E000041E0BD1074B1B68002B07D068782A7863
:1056F0000002104342425041013098472000FEBD55
:1057000002290000885EFF1F30B5012503790400DF
:10571000BFB02B4225D01449408805F05BF82842E1
:105720000CD0124B01A95B8D00220B8002234B8011
:105730000F4B5B888B80608802F042F90D496088CE
:1057400005F048F8C0070CD50B4B01A91B880022B7
:105750000B8002234B80064B9B888B80608802F075
:105760002FF93FB030BDC046805EFF1FAC3CFF1F2D
:10577000145CFF1F785EFF1F063DFF1F10B5074C2E
:105780000749200004F0DCFF2000064904F0D8FFA0
:105790000721054A054804F095FF10BDFFFF0000F2
:1057A000805EFF1F785EFF1F34B90011AC3CFF1F05
:1057B00010B5024802F086FF10BDC046095700111F
:1057C0000200F0B501270A480A4E51188B1A002B27
:1057D00000DCF0BD082415784308684038404000DC
:1057E000805B013C58406D08002CF5D10132EDE79B
:1057F000FFFF00004EB90011F0B500250F269D42B5
:1058000000DBF0BD4C5D070944403440A400A058C3
:1058100001357840F3E70000F0B589B06A460D0025
:105820000B000F27110010351C78013326002409C6
:105830003E40167054700232AB42F5D12023024A2A
:10584000FFF7DAFF09B0F0BD54B90011F0B54E789A
:105850000B7889B036020C00170001901E43012A14
:1058600061D9954B9E4200D877E001339E421CD10E
:10587000062A17D1CA788B7812021A430B791B04B7
:1058800013434A7912061A438C4B5A6100221A704C
:105890005A808B4A5A608B4A9A608B4ADA600020A1
:1058A00009B0F0BD88225205EEE7884B9E423CD1FC
:1058B00082498B78002B00D0F6E00C2A31D10F22E0
:1058C000A3789343E278120213432279120413431C
:1058D0006279120613434B60E279A0791202024307
:1058E000207A00041043627A12060243CA60E27A08
:1058F000A07A1202024376484A81834208D80423E0
:105900006E49142201980B7005F036FF1420C7E78A
:105910001201D21889235B059A42F0D801238B70BB
:10592000BDE7022AFAD00523EAE76A4A0123964234
:10593000E6D1FFF705FC052F0CD9E378A2781B020E
:105940001343227912041A4363791B061343624AF4
:105950000393136005F020FFA1E7584D2B78002B2F
:105960009DD1AB78002B00D1A0E02B8901339BB2F5
:105970000093B34200D091E0132AD4D9CF7C8B7C22
:105980003F02122120001F43FFF71AFF874200D079
:105990008EE0002E3DD1E378A2781B0213432279DA
:1059A000E96812041A4363791B06134303930A221E
:1059B0008B4212D1FF23A370E370237163716B8953
:1059C000002B09D1E37B227C1B0212041343A27B30
:1059D00013431B0901336B8100226B89002B8ED08E
:1059E000002A67D1686837013818000B6B6900031B
:1059F0000390984205D9686105F0F6FCEB78013315
:105A0000EB7068681022A11C381805F01DFD2E816E
:105A100045E76F89009A7B1E9BB293423AD1E278A8
:105A2000A37812021A43237905A81B041343627951
:105A30006C6812061A43EB6800920392211D0C2237
:105A4000049305F099FE0120260004A94042103677
:105A5000FFF7E2FE013F012F17D1009A0B232861C7
:105A6000824200D04CE704221C49200005F0ECFCE7
:105A7000042203A9686805F0A7FBE968039AFF23DD
:105A8000914200D13CE7F73B3AE73100FFF7C4FE13
:105A90001036DFE70923B742A4D831E7009BB342B1
:105AA00000D9FCE607232BE7022329E7032327E796
:105AB000062325E70A2323E7FFFE0000203DFF1F02
:105AC00000000111FFFF00005048593601FF00009F
:105AD000FFFF001102FF000034F000402C3DFF1FCB
:105AE00010B5034C0B000122210000F06BFA10BD31
:105AF000A15C00110B8870B506000D000224162B66
:105B000011D92B000322094900F05CFA041E0AD1C6
:105B1000074B2A881B88191C934200D9111C30009E
:105B200089B200F0EFFA200070BDC046CD5C0011D4
:105B3000B25EFF1F10B54A780400013A0B00022044
:105B4000012A07D80A78002A04D005222000024939
:105B500000F038FA10BDC046FB5C00110A7810B5A1
:105B60000B0004000220002A04D007222000024972
:105B700000F028FA10BDC046A75D00110A7810B5E4
:105B80000B0004000220002A04D009222000024950
:105B900000F018FA10BDC0460D5E001110B5034CA0
:105BA0000B000B22210000F00DFA10BD3D5E00112C
:105BB00010B5034C0B000D22210000F003FA10BDBC
:105BC000AF5E001110B5034C0B000F22210000F056
:105BD000F9F910BD095F00110A7810B50B00040037
:105BE0000220002A04D011222000024900F0EAF924
:105BF00010BDC046195F0011002310B51322190013
:105C000000F0E0F910BD000010B5034C0B001722A6
:105C1000210000F0D7F910BD6B5F0011002310B513
:105C20001922190000F0CEF910BD000010B5034C88
:105C30000B001B22210000F0C5F910BDA55F00116B
:105C4000F7B584890D0006000121002C22D0002325
:105C50008268D3561778002B1EDA0C2C1AD90C3C0C
:105C6000A4B2131940880093230002F086FE431E5D
:105C7000984101307B06DB0F6B703F23013C1F40D6
:105C8000A4B22870AF70AC80002C07D0B368013389
:105C9000AB6000210800FEBD0020EBE7AC60F8E738
:105CA0000B7803704B8843704B881B0A83700B7909
:105CB000C370042070470420022B06D100205378C3
:105CC00011781B02009A0B43138070470B880370F6
:105CD0000B881B0A437002207047042000998342FE
:105CE0000AD1537810781B0203430B80D378907845
:105CF0001B02034300204B807047F8B50D004B7822
:105D000001240021461C03702B788B4201D820000F
:105D1000F8BD6B78B01C4F1C012B10D1890069189D
:105D20004B88022233704B88B9001B0A73706918C4
:105D300005F062FA04360434A4B2F9B2E4E712239F
:105D400059436B185A88043132705B8810221B0A41
:105D50007370691805F050FA12361234ECE770B51A
:105D6000049D14001E00052B01D8042070BD63782B
:105D700012781B0213432B80E378A2781B02134393
:105D800002226B802A71211D681D063E05F034FA3F
:105D9000B2B22A81E92AE8D82800A11D0A3005F00C
:105DA0002BFA0020E2E7002310B50A789A4201D8C6
:105DB000900010BD9A008A185488013304705488EA
:105DC000DBB2240A4470948884709288120AC270EC
:105DD0000430EAE710B51100029C062B04D0042021
:105DE0001022142B01D010BD022222714B780878AA
:105DF0001B0203432380CB7888781B020343638014
:105E00000431601D05F0F8F90020ECE710B50C78BE
:105E10008B7804315C43E4B203702200013005F05A
:105E2000EBF9601C10BD0420022B06D10020537832
:105E300011781B02009A0B431380704710B50C00B9
:105E40000A88023105F0D8F9208810BD70B5040029
:105E50000D0004981100012B01D8042070BD1678A4
:105E600052781202324302800200F13255701470EF
:105E7000E125002C00D10C35023B9AB24280AA42A7
:105E8000EBD80231043005F0B7F90020E6E7042032
:105E9000009983420AD1537810781B0203430B8088
:105EA000D37890781B02034300204B80704710B5D5
:105EB0000C000A88023105F09FF9208810BD00000F
:105EC00070B501211E000420049C0E400B4218D125
:105ED000CB40DDB28D4214D90A49DBB20988994220
:105EE0000FD32300EE331D7033005800111849788A
:105EF000165C0902314301332152D9B28D42F4D8E4
:105F0000002070BD383DFF1F10B50C000A8802311B
:105F100005F072F9208810BD10B50C788B7804312B
:105F20005C43E4B203702200013005F065F9601CA7
:105F300010BD10B511000298032B01D8042010BD2C
:105F400014785278043B120222430280CA788C787B
:105F50001202224342809AB28280EB2AEED80431A8
:105F6000063005F049F90020E9E710B50C000B8870
:105F700003700B881B0A43704B8883704B881B0A85
:105F8000C3708A880430063105F036F9A0880430E1
:105F900080B210BD0420012B03D100201378009A99
:105FA0001370704710B50C000B8803700B881B0A28
:105FB00043704A880230043105F01EF960880230CF
:105FC00080B210BDF0B589B003931E4B029242001F
:105FD0000700D05A019102F020F81325061E2DD09B
:105FE000029B01240370019B002B04D0001903992C
:105FF0009847001984B26B461B7A5BB2002B0FDA0C
:106000001021380002F01CFB1925002813D13000A4
:106010003219E1B202F066FC051E0CD10C34A4B2B8
:10602000042304AA380005A993800696948101F000
:10603000AFFD051E02D0300005F076FA280009B049
:10604000F0BDC046B05EFF1F70B505000C00002813
:106050000CD00020814209D010222000044905F014
:10606000CBF801202B7823736B78637370BDC04627
:1060700094B90011F0B506000D0017001C0085B0A2
:1060800002291BD00020102907D1022B07D0102B8A
:1060900003D115E00020102C08D005B0F0BD6946F2
:1060A0003800FFF7D1FF2A0069460BE0694630004F
:1060B000FFF7CAFF22006946380004E0022BE9D14D
:1060C0002A003900300005F0EFF9E6E7031CF0285C
:1060D00000D9F023032008499AB2013A0B80D31764
:1060E000034006499B189B100B80D30F04499B1853
:1060F0005B100B807047C0463C3DFF1F3A3DFF1FC1
:10610000383DFF1F034B1B888B4202D3024B4000DC
:10611000C15270473C3DFF1FB05EFF1F014B400066
:10612000185A7047B05EFF1F1722014B1A80704744
:10613000B05EFF1F70B505000E2005F0BDFA041E0D
:1061400013D0D023037000230622837007494570C3
:10615000033005F051F8064B2100DA8A62811B7E7C
:106160002373044B187805F01FF970BDCC5EFF1F38
:10617000BC5EFF1F8C3DFF1F262803D8024B40004A
:10618000C05A70470148FCE73E3DFF1FFFFF00007B
:1061900070B506000C00094D1C220021280005F0F6
:1061A00043F8074B1E70074B1C7005F0D5F901230F
:1061B000002801D0002312202B7070BDBC5EFF1F91
:1061C0008C3DFF1FDD5EFF1F70B505000D4C080004
:1061D000E260A16010220021656005F065F80128E9
:1061E00003D11021A06802F058FD102200212800E0
:1061F00005F05AF8012803D11021606802F04DFD26
:1062000070BDC046BC5EFF1F70B5041E05D10029DD
:1062100003D006220D4804F0EFFF0D4B1D78012D31
:1062200011D1002C05D102221A7005F025FA2800A0
:1062300070BD00221A70074B1B78FF2BF7D020008F
:10624000FFF778FFF3E70025F1E7C046CC5EFF1FBC
:10625000BC5EFF1F8C3DFF1F030010B5002801D15D
:10626000002010BD00780B4A002803D15988D18244
:106270001B7913761378022BF2D10023984200D1B8
:1062800003331370044B1B78FF2B01D0FFF752FF31
:106290000120E6E7BC5EFF1F8C3DFF1F002911D0E7
:1062A00000280CD04B79012803D1402252421343DD
:1062B00003E03F221340032802D001204B717047B6
:1062C0004022F4E70800FAE770B5094D010028788C
:1062D00000280BD0074C0622200004F08DFF21007F
:1062E0002878FFF7DBFF200005F00EF970BDC046EF
:1062F000DC5EFF1FB65EFF1F00290AD0012808D10F
:106300003F224B799343C02B03D0403B5A42534129
:10631000981C704770B5174D06002B78FF2B15D0D1
:106320000A2005F0C9F9041E10D0D0230370C83B21
:106330008370114B11491B784670C37006220430DC
:1063400004F05AFF2100287805F02EF80C4B1B783A
:10635000012B0DD10B4B1B68002B03D09B68002B2E
:1063600000D09847084B04211878084A05F064F8D3
:1063700070BDC0468C3DFF1FDC5EFF1FB65EFF1F79
:10638000D85EFF1F045FFF1F085FFF1F60EA000069
:10639000014B98687047C046BC5EFF1F014BDB682D
:1063A00018687047BC5EFF1F074B10B5DA681368AA
:1063B00001331360054B1878FF2803D08021C901F1
:1063C00005F05AF810BDC046BC5EFF1F8C3DFF1F94
:1063D000F7B50E0002F0C8F8051E1CD00E4B066281
:1063E0001F78002F00D10778AB791020019305F0BA
:1063F00063F9041E0FD0D0230380C73B8370019B39
:10640000E91DC3700622043004F0F6FE21003800B6
:10641000E66004F0C9FFF7BD8A3DFF1F014B187805
:106420007047C046DC5EFF1F054B002805D1054BB9
:106430001A78054B002A00D1014B18007047C0465E
:10644000CC5EFF1FDC5EFF1FB65EFF1F014B58686E
:106450007047C046BC5EFF1F024B1868431E984140
:10646000C0B27047E05EFF1F421E03000120152AE4
:1064700003D9FF3B5A425341D8B27047F0B51C00D4
:1064800000230E0085B0039002920B70029A934293
:1064900001D3002019E0E55C5A1CD2B2002DF8D0DF
:1064A000029851198142F4DC0233DFB2A35C180078
:1064B0000193FFF7D9FF002807D0013D019A039906
:1064C000EBB233708A4202D1E01905B0F0BDDB199E
:1064D000DBB2DBE710B50C0002F09EF803001220DF
:1064E000002B03D02100588804F006FF10BD0000E7
:1064F00070B50E4D84006359002B15D0186A002822
:1065000001D005F0D1F82B59586A002801D005F0C8
:10651000CBF82B59986A002801D005F0C5F8285906
:1065200005F0C2F800232B5170BDC046EC5EFF1F82
:106530001C4B70B504000E00150099420AD11A4B8D
:106540001B68002B01D1122070BD1B68002BFAD0F4
:106550009847F9E7154B994215D1134B1B68002B4F
:106560000AD01B68002B07D09847002804D1104B95
:106570001C70104B1D70E7E729002000FFF7AAFFF1
:106580000028E1D1F3E7080001F0EEFF0028DAD09F
:1065900003780320A342D7D12900300004F0ACFED9
:1065A000D2E7C046FEFF0000E85EFF1FFFFF0000CD
:1065B000E55EFF1FE45EFF1FF7B50400808801F071
:1065C000D3FF0025A84203D00578A08802F008F880
:1065D0001C4E3378002B1FD0AB421DD11A4B280024
:1065E0001978FFF777FF002818D000233370A379BC
:1065F0000820A778A688019305F05EF8011E0DD04B
:10660000D0230370CA3B8370019B477086808371DF
:10661000280004F0C9FE01E0002DE8D1A0880B4B52
:106620008200D358002B01D0FFF762FF1721A0880A
:10663000FFF768FDA08801F027FDA08801F0FEFDAE
:10664000F7BDC046E55EFF1FE45EFF1FEC5EFF1F67
:10665000F0B587B01D000CAB1B88070001930DAB94
:106660001B88142002930EAB1B88160003930FABFC
:106670001B880091049310AB1B88059305F01CF850
:10668000041E1AD0D0230370CB3B47708370C670B2
:10669000062229000430002D11D004F0ADFD019B2D
:1066A00021006381029B0098A381039BE381049BEB
:1066B0002382059BA37404F077FE07B0F0BD04F0BD
:1066C000B3FDECE7F7B5009308AB1B8807000C207F
:1066D0000D001600019304F0EFFF041E13D02800F4
:1066E00001F042FF00280FD00078D0232370C93B6F
:1066F000A370009B21002381019B6770A580E68029
:10670000638104F051FEF7BD014B1878EDE7C046F8
:106710008C3DFF1F13B5040064890389C2888188FA
:10672000C0780094FFF7CEFF13BD000010B5044CF5
:106730002068002803D004F0B7FF0023236010BDB9
:10674000F05EFF1FA122F0B5818892004A43384BCA
:10675000384F1B6804009B189D2292009B18827979
:1067600089B01A603B68002B5FD01D78324B1B68E4
:10677000002B04D05B68002B01D000209847260036
:1067800008363100E079FFF7B7FD237DE0710200A4
:10679000E0780493638A29000393238A0293E389B0
:1067A0000193A38800933300FFF752FFE378002B97
:1067B0000BD1E289A379A18802920196E27928009F
:1067C0000092012201F0DAFEE0703B68002B20D03D
:1067D000FFF7ACFF194D287800281AD0184B19780C
:1067E000FFF778FE002814D02B78E678082007936E
:1067F000A78804F061FF011E09D0D0230370CA3BB3
:106800004670837087808671079804F0CDFD002361
:106810002B701721A088FFF775FCA08801F034FCCD
:10682000A08801F00BFD09B0F0BD064B9DE7C04606
:106830003409FF1FF05EFF1F045FFF1FE55EFF1FAF
:10684000E45EFF1F8C3DFF1FF8B5070008000E0037
:1068500001F08AFE041E18D02620FFF78DFC051ECD
:1068600000D12578062004F027FF041E0DD000215A
:10687000062204F0D9FCD0232370C23B21006770AC
:10688000A370A680E8B204F08FFDF8BDF0B585B026
:1068900001930AAB1B78070002930BAB1B7808002F
:1068A0000D000092039301F05FFE061E22D010201F
:1068B00004F002FF041E1DD01022002104F0B4FCDD
:1068C0002620FFF759FC002800D13078D023237010
:1068D000C13BA370009B21002372019B6770637210
:1068E000029BA580A372039BC0B2E3720C9BE36082
:1068F00004F05AFD05B0F0BDF7B50D00019001F0B0
:1069000033FE071E20D00E2004F0D6FE041E1BD03E
:106910002620FFF731FC061E00D13E78D0232380CD
:10692000C53B0622A370F91DE01C04F065FC019B29
:106930002A0063810123DD401A401D40210022739B
:106940006573F0B204F030FDF7BD0000F0B585B01E
:10695000029010000D0017000A9E039301F004FE40
:10696000041E31D0029B002B2ED1039B02795B07C2
:1069700024D5122313430422002E08D10B99002999
:1069800005D10C99002902D10D9900291AD01A437A
:106990000D9B2271002B00D0C9E0002E00D1CFE06A
:1069A000002D00D0CCE0606A002801D004F07CFE0D
:1069B0001C21300004F030FD606205E002239A43A0
:1069C0000E33D7E793432371654BBA00D458002C9C
:1069D00000D1AAE0002E10D0236A002B03D11C2086
:1069E00004F032FE20625E4BBA00D358186A0028C9
:1069F00003D01C22310004F0FFFB0C9B002B12D0B3
:106A0000574CBB001D596B6A002B03D1162004F0B4
:106A10001BFE6862BB00E358586A002803D01622A8
:106A20000C9904F0E9FB0D9B002B11D04C4DBC00E0
:106A30006659B36A002B03D1142004F005FEB0623E
:106A40002B59986A002803D014220D9904F0D4FB26
:106A5000380001F089FD051E67D0414BBA00D358BC
:106A6000002B62D01A6A3420002A00D11C389A6A9E
:106A7000002A01D0143080B20B9A002A01D01C30B9
:106A800080B25B6A002B01D0163080B204F014FE95
:106A9000041E4AD01822002104F0C6FB2620FFF76E
:106AA0006BFB0190002801D12B780193D023237038
:106AB000029B200063700A23294EA370039BBD0034
:106AC000A371AB59A780196A1830002905D01C2280
:106AD000A06004F091FB200034307359996A0029BA
:106AE00007D0030014221433E060029304F084FB07
:106AF00002980B9B002B08D003001C221C330B991F
:106B00002061029304F078FB02987359596A0029B6
:106B100003D01622606104F06FFB6B4621001879E8
:106B200004F042FC3800FFF7E3FC05B0F0BD102292
:106B30000D9B0D991B69A018236204F05DFB2CE7E7
:106B40000B9B002B00D13FE7012D00D03CE7606A92
:106B5000002801D004F0A8FD1C210B982AE7C046AC
:106B6000EC5EFF1F10B5044C2068002803D004F031
:106B70009BFD0023236010BDE05EFF1F0B4B07B59C
:106B80001A68002A01D100200EBD6946531C01205D
:106B900012780731FFF772FC0028F4D00278012345
:106BA000100018401A42EED0EEE7C046FC5EFF1F10
:106BB000F0B51F4F01203B6887B0002B25D09B7894
:106BC000059300F0B3FB002821D00A20FFF7D4FA88
:106BD00004000B20FFF7D0FA164B05001E78731E39
:106BE0009E413B68F6B2191DD878FFF757FB3B680A
:106BF0002900DA7A043303929A7901930292009081
:106C000033002000059A04F05FFD07B0F0BDFFF7E8
:106C1000B5FF002805D00620FFF7AEFA04000720D4
:106C2000D8E70820FFF7A8FA04000920D2E7C046F9
:106C3000E05EFF1FDC5EFF1F70B50A4E0400337874
:106C40000D00FF2B0DD0042004F036FD011E08D0EE
:106C5000D0230370CE3B45708370C470307804F04D
:106C6000A3FB70BD9C3DFF1F70B5040006200D0006
:106C700004F022FD011E0AD0D0230370CD3B8370A7
:106C8000054B44701B688580187804F08DFB002C40
:106C900001D0FFF767FF70BDE05EFF1FF8B5264F1C
:106CA00006003B680D001124002B05D10522234B63
:106CB0001B78134202D112242000F8BD204A102470
:106CC0001268002AF8D01278002AF5D0DB0719D50F
:106CD0002B789A1E012A1AD80C2004F0B5FC132434
:106CE00038600028E8D000230A224370290006708B
:106CF000023004F081FAFFF75BFF041E0AD0FFF7B1
:106D000031FFD9E700F012FB0028E1D1E4E7002BC6
:106D1000E2D0D0E70B4B1B78032BCDD11D20FFF722
:106D20002BFA094B18800028C6D0084B042118788C
:106D3000074A04F081FBBFE7E05EFF1FDD5EFF1F37
:106D4000FC5EFF1FDC5EFF1FDA5EFF1F085FFF1F98
:106D500060EA0000F7B50193194B14001A78052377
:106D600006000F0012201A4221D0012920D1154B14
:106D70001D68002D1BD002201F2C18D8002C02D01B
:106D8000019B002B13D0104B1F221E706E1C002184
:106D9000300004F049FA01992200300004F02CFA86
:106DA000310020002C70002F06D004F0ADFAFEBD9B
:106DB000064B12201D68DCE704F066FBF7E7C046CF
:106DC000DD5EFF1FFC5EFF1F9C3DFF1FF85EFF1F87
:106DD000F8B50F4E12243368002B17D01B780F3CE8
:106DE000834213D100250B4F0221387804F0ECFCCC
:106DF000094B042138781D8004F0E6FC074B28007D
:106E00001D8033685C7004F0A7FA04002000F8BD10
:106E1000E05EFF1F085FFF1FF45EFF1FDA5EFF1FCB
:106E200070B5012823D11B4C2388002B03D01A4AAC
:106E30001578002D07D0194B1B68002B02D018784D
:106E4000FFF7C6FF70BD3B2B02D93C3B2380F9E71F
:106E5000134E0221307804F0B7FCFA222388920006
:106E600002215A43307804F0CFF92580EAE70B4B32
:106E70001B68002BE6D00B4B1B785B07E2D5084B59
:106E80000221187804F0A0FC0022024B1A80FFF7C0
:106E900069FED7E7F45EFF1FD85EFF1FE05EFF1FAD
:106EA000085FFF1FDD5EFF1FF8B51E4D2868002834
:106EB00003D004F0F9FB00232B601B4E3068002840
:106EC00003D004F0F1FB00233360184F05243B7816
:106ED00018002040234221D0154800F02BFA3B78BF
:106EE000234213D0202004F0AFFB2860002813D0E9
:106EF0002022002104F098F9202004F0A5FB041EB4
:106F0000306005D02022002104F08EF9002004E03A
:106F1000286804F0C9FB2C601320F8BD00F00AFAC1
:106F2000F4E7C046FC5EFF1FF85EFF1FDD5EFF1F3B
:106F3000903DFF1F10B50A4C23681A1E0ED0002882
:106F400008D10130587004F007FA002805D02368F2
:106F5000002B02D00021FFF787FE0122100010BD98
:106F6000E05EFF1FF7B5274E050033680191181E3C
:106F700021D05C78244F012C30D1FFF7FFFD002891
:106F800025D02000FFF7F8F80400412814D91F4B42
:106F9000022118781E4A04F04FFA1E4B3C3C1C801C
:106FA000022233685A703B78002B14D128000199D3
:106FB000FFF75AFE0120FEBDFA2292004243002A4A
:106FC000EED0124B0221187804F01EF9E8E7FFF723
:106FD000D3F80200F3E700233B70EBE73B78002B8C
:106FE000E8D1032004F068FB011E08D0D023037011
:106FF000CC3B457083703368187804F0D5F9FFF7FF
:10700000B1FDD7E7E05EFF1FD85EFF1F085FFF1FDF
:1070100060EA0000F45EFF1F10B517498388020084
:107020008B4220D011D815498B4217D0144900202B
:107030005B1899B2012907D8926811785A425341D6
:10704000D8B2FFF7F9FD012010BD0E4A00209B18B1
:1070500007229BB29A424041C0B2F5E78368187894
:10706000FFF768FFF0E7836899785A780902187883
:107070001143FFF777FFE7E70A2000000620000032
:10708000F8DFFFFFAFDFFFFF014B18707047C0460E
:107090009D3DFF1F10B5064C207001F041FA20788D
:1070A00004F092F90521207800F062FD10BDC04681
:1070B000085FFF1F0BB273B50D00002B00DBC4E0AF
:1070C000884B187804F0B0FA041E0ED00378912B88
:1070D0000FD0A22B00D1A1E0834B1878FF2852D00B
:1070E000210004F061F900284DD1802000026840A1
:1070F00076BD43780F2B76D013D8052B70D00E2B8E
:10710000EAD18088794B98422BD8794B98421BD88A
:10711000784B9842E0D1A3681878591CFFF774F8AF
:1071200038E03E2BD8D18378032B74D06CD8012B58
:107130006ED0022BD0D1704B1B68002B23D05B6824
:10714000002B20D098471EE06C4BC0180C28C3D8E9
:1071500004F042FB1DC2C2150BC20B0B0B3223C243
:107160003C00674BC0180728B6D8664B1B68002B3D
:1071700009D01B68002B06D0200098470AE0A368BE
:107180001878FFF7C7F8200004F0AEFAADE7A06862
:10719000FFF762F800289FD0F5E7A3681B78002B63
:1071A000F1D0554B1B68002BEDD01B68002BEAD0AB
:1071B000210055489847EDE74F4B1B68002BE2D064
:1071C0001B68002BDFD021005048F3E7504B1B68B1
:1071D000002BD8D05B68002BD5D021004348E9E7CD
:1071E000FFF7EAF9CFE780884A4B984203D04A4B31
:1071F000984200D070E7464B1B68002BC3D05B68F9
:10720000002BC0D02100D5E7153B012BBBD963E78C
:10721000FFF798FAB7E7FFF77DFAB4E73F4B1B7823
:10722000042B07D100236A4613800179408800F0BF
:10723000C5FCA8E7364B1B68002BA4D05B68002B6D
:10724000A1D00100364898479DE7012421420AD089
:10725000294B1B68002B04D05B68002B01D0002059
:107260009847012043E78B070AD5264B1B68002B64
:1072700004D05B68002B01D020009847022036E73D
:107280000421280008400D4200D131E7254E338803
:10729000002B21D0013B9BB23380002B1AD1FFF78A
:1072A000DBF800280AD0204B1C70164B1B68002B03
:1072B00004D05B68002B01D020009847FFF7C6F888
:1072C000694601F001FD6846FEF7FEFF1D20FEF74E
:1072D00053FF308004200AE7024B187804F074FA58
:1072E000F8E7C046085FFF1F9D3DFF1F0E2000000E
:1072F0000120000009100000005FFF1FFEDFFFFFFC
:10730000AFDFFFFF045FFF1F0C2000000B20000019
:10731000E85EFF1F0D20000013200000DD5EFF1F50
:10732000FFFF0000DA5EFF1FD85EFF1F10B501F0FF
:107330009BF910BD014B18607047C046045FFF1FEA
:107340000B880020162B01D817230420014A138034
:107350007047C046B25EFF1F00207047074A030017
:107360001188814207D091880020994202D10130D2
:107370008000101870470020FAE7C046105FFF1F1A
:10738000F0B58F7806000D00C5B01E2F15D1FFF7A0
:10739000E5FF051E03D10024200045B0F0BD00220A
:1073A0003B003100C078009200F0B2FB0400A81C42
:1073B00000F0D2FBFF23EB70EEE7264B062403938D
:1073C0001B78FF2BE8D0182FE6D87B08224A013B18
:1073D000DB0002929A589446002ADDD0029AD31814
:1073E0005B68002BD8D00878002802D14B78012B9D
:1073F00002D10624122FCFD107AFAB88697800974E
:107400006446AA68A047041EC6D1AB78029A5B08FE
:10741000013BDB00D318390030005B689847041E3D
:107420000BD1AB78042BB6D0039A31001078220030
:10743000009700F06DFB0400AEE76A78002AABD13C
:10744000AA7805A93B88087130000A704B80FEF7C6
:1074500047FBA0E7A03DFF1FA4B900111D4B37B5A6
:10746000050098420BD000290AD1FFF777FF0028CA
:1074700005D11948FFF772FF002800D0058037BDFD
:1074800001291AD1FFF76AFF041EF8D001235B42DD
:107490000380A378FF2BF2D0FE2B07D00023E078E7
:1074A0001422009329001E3300F032FBA01C00F0D0
:1074B00053FB01235B426380E1E70229DFD10139FD
:1074C00001F0BEF80028DAD12800FFF747FF041EBC
:1074D000DFD1D4E7FEFF0000FFFF0000022210B55D
:1074E000074B52421A80074801325A809A80DA804C
:1074F00000F07EFA044801F025F8002010BDC046D7
:10750000105FFF1F817300115D7400110388F7B5D0
:107510000400002B02D102252800FEBD4268022192
:10752000137825485268FEF7A5FD00282ED0234F7A
:1075300001253A88002AEFD0802321885B020125AB
:107540009B1A9942E8DC0C2004F07EF8061E31D02C
:107550003B8822889C4600231800019561469DB215
:10756000491989B2AA421BD8002801D062443A8046
:1075700000233000082208C0210003F03DFE104A1D
:107580001368002B13D100251660C5E7626802213D
:1075900013780C485268FEF76DFD0028C7D1BAE792
:1075A00060681D014019418101330198D6E71A0036
:1075B0001B68E6E71325AFE712BA00119E3DFF1FD7
:1075C0000C5FFF1F10BA0011014B18707047C046C6
:1075D000A03DFF1F14230A0010B51A40194204D021
:1075E0000122102101F048F810BD4B06F9D401200A
:1075F00088434000F8E710B514008B0604D501223B
:10760000102101F039F810BD08230A001A40194270
:1076100002D14BB2002B0FDA102101F02DF8002817
:1076200008D02300F2331B78002BECD0F134237800
:10763000012BE8D10020E6E703208907FAD4E2E72E
:10764000F0B51F00184B85B01C68019002910392A1
:10765000002C27D1200005B0F0BDA5683301ED183E
:107660006B89019A934211D3029A93420ED8002F4C
:1076700004D10A9B002B10D12C00EBE73B002978AA
:10768000039A6868FEF7F6FC0028F2D10136B6B21C
:10769000A388B342E1D82468DAE7A3680A9A5B8931
:1076A0001380E9E70026F3E70C5FFF1F37B50C00F6
:1076B0000A8849880123914217D3002A15D0651DF5
:1076C00023792A0002210A48FEF7D4FC102300285F
:1076D0000BD023796188208800242A000094FFF7CA
:1076E000AFFF0A23A04200D0230018003EBDC046D1
:1076F00012BA001113B50A0008884988012388428C
:107700000BD8002809D00024137905320094FFF724
:1077100097FF0A23A04200D02300180016BD13B51E
:107720000A0008884988012388420BD8002809D01C
:107730000024137905320094FFF782FF0A23A04248
:1077400000D02300180016BDF0B58BB003904A8816
:1077500008880E000123824255D3002853D000230D
:10776000012704AC23700022718813000092FFF7F8
:1077700067FF051E3ED02078002835D12B78022BDC
:1077800018D167706A8983000130E31880005A803D
:1077900069680222201803F02FFD23780133DBB241
:1077A0002370042B19D93B006889013080B2002B6B
:1077B000D9D01FE002236370122358436A8923182B
:1077C00004305A8069681022201803F015FD2378D0
:1077D0000133DBB22370002BE5D10C4A6B899B1877
:1077E0005A425341DBB2DFE76378012BE4D12B78B7
:1077F000022BC7D022780A23002A04D02100039844
:10780000FEF798F9002318000BB0F0BD0100FFFF50
:107810000F4BF0B504001868002816D083685D8906
:10782000A54207D88288AE18B44203DA12019A182A
:10783000934201D10068EFE71E005F891036A7422E
:1078400004D1002900D00D801800F0BD3300EFE70F
:107850000C5FFF1F70B505000C0008880021FFF7C2
:10786000D7FF03000120002B04D022002800197A42
:10787000FFF7C1FE70BDF7B50C0000250190230095
:10788000EE331B78AB4201D800200AE06B00E65AC9
:1078900000213000E718FFF7BBFF002802D1268047
:1078A0000130FEBD017A0198FFF794FE002802D056
:1078B0003B882380F5E70135EDB2E0E710B5040021
:1078C00008880021FFF7A4FF03000120002B03D04C
:1078D0002000197AFFF77EFE10BD0000054B1B68E3
:1078E000002B01D1180004E09A6852898242F6D137
:1078F000988870470C5FFF1FF0B50E27002687B0F1
:10790000039302ABFF183E8005001F4B4089140013
:10791000984207D02B78013000976A6880B2FFF751
:107920008FFE060002212B7818486A68FEF7A2FB3A
:1079300000280FD06C892000FFF7D0FF002802D06C
:10794000013C0419A4B2039B002B00D01C80300022
:1079500007B0F0BD02212B780D486A68FEF78AFB5C
:107960000028E7D102212B780A486A68FEF782FBDB
:10797000002807D0002EDED03B88A342DBD17489DB
:10798000013CDFE76C89DEE7FFFF000012BA00115F
:1079900010BA00110EBA001110B50C00FFF7DEFC92
:1079A00003000220002B0AD0002C00D023609B781B
:1079B0001720FE2B03D00138FF2B00D1002010BD73
:1079C00073B50D0001A904001600FFF7E5FF1728A5
:1079D00005D0002E04D129002000FEF727F976BD3E
:1079E00001221021200000F047FE0028F3D0F6E726
:1079F000014B18607047C0461C5FFF1F37B56B46D0
:107A00009D1D010004000222280003F0B5FE2B8812
:107A1000B02B0ED12379122B09D12300FA331B7816
:107A2000012B06D10121608800F0E0F801E01B2B5A
:107A3000F8D037BD10B5054B0421187000F098F848
:107A4000FFF74CFDFEF770FB10BDC046205FFF1F27
:107A50000020F0B50BB20F0087B0834234DA274B19
:107A6000187803F0E1FD051E2BD00378A02B25D15B
:107A700003AE3100FEF7E4F8041E0BD1B378DB0748
:107A800024D51F4B06341B68002B03D031006888B7
:107A900098470400A868002801D003F045FD002C99
:107AA00008D1184A039B1340174A934206D0B37873
:107AB0001B2B03D00121688800F098F8280003F000
:107AC00013FE80200002784007B0F0BD0F4B1B680A
:107AD000002B10D0310068889847041EDAD07378E4
:107AE000002BD7D1B27801A90A704B800C7168883D
:107AF000FDF7F6FFCEE70624F1E7C046205FFF1F43
:107B0000185FFF1F00FFFF00000112001C5FFF1F36
:107B1000F7B50190FC200D0017001E0003F0CCFD0E
:107B200004001320002C12D0B02320002370089BE7
:107B3000F4226770658026710830002B08D0190088
:107B400003F05AFB2100019803F02EFC0020FEBD3B
:107B5000089903F069FBF5E710B5041E06D000781C
:107B6000FD2803D803F048FEFF23237010BD00005A
:107B70000A1F93B210B504000220032B05D88240DF
:107B80000020024BD1529B189C7010BD405FFF1F1C
:107B90000B8870B5043B04000D000220032B0BD8AA
:107BA0000121200000F04CFD03001420002B03D025
:107BB0002900200000F0DEFB70BD000007B51300B7
:107BC000034A00920A00012100F02CFC0EBDC046C1
:107BD000F97D001107B5019203220092024B0A00C1
:107BE000122100F049FC0EBD777E001107B56B46EF
:107BF00001AA11800449D88008780633012802D1EF
:107C0000190003F011FC07BD215FFF1F0C4B10B5DD
:107C100018700023FF210B4A1380138193819380F6
:107C2000094A53801370517293819372D174D38235
:107C30001375517703F0A8FB00F0FCF910BDC046A6
:107C4000505FFF1F405FFF1F225FFF1FF0B58DB029
:107C50006B46002003910C229B5E834200DBB0E068
:107C60005D4B187803F0E0FC051E00D1A4E003781A
:107C7000902B00D09DE006AF01004688380000F050
:107C800013FA79680400002900D19CE03B88052B99
:107C90006ED13B89032B1CD905AC200000F0A2F863
:107CA0006288172A61D83989131D994231D17968C0
:107CB000237804310291D90738D5607800F08EF925
:107CC000071E06D0002303712378012B08D0132B45
:107CD00023D0A868002800D178E003F025FC75E0E7
:107CE0006288029909A800F0A6F80290380000F016
:107CF0008BF909AA2378387A019200223100009288
:107D0000029A00F012F9380000F064F9029B002B8F
:107D1000DFD0300000F080F9DBE70378032BD8D107
:107D20006288029909A800F0D6F8DEE7122B13D179
:107D3000029909A800F0B5F8021EEAD127498B88FC
:107D4000002BC6D0887909A9237801916178009128
:107D5000310000F0EAF8BCE7002302AA9383300068
:107D6000617809AAFFF72AFFB3E71D4B0993F6E7ED
:107D7000042B02D09A1F012AABD8184A043B9B005F
:107D8000995A0029A5D0D218907831003A0000F015
:107D9000AEF800289DD13B88042B03D00121300090
:107DA000FFF724FF012C04D1A868002801D003F0BC
:107DB000BBFB280003F098FC8020039B000243409B
:107DC00018000DB0F0BD012800D182E7012130007C
:107DD000FFF70CFFEDE7C046505FFF1F405FFF1F3E
:107DE000010017000B7803704B784370CB788A78CA
:107DF0001B021343438070470A88030002700A88FD
:107E0000120A42700A88012A06D14A8882704A887A
:107E1000120AC2700420704702208242FBD14A88B5
:107E200004309A704A88120ADA708A881A718A882D
:107E3000120A5A71EFE710B50400012082420CD9F2
:107E40004B780A781B0213432380834206D1CB78F8
:107E50008A781B0213436380002010BD022BFBD1E4
:107E6000CB788A781B02134363804B790A791B0213
:107E70001343A380F0E70B8803700B881B0A437041
:107E80004B8883704B881B0AC3708B8803718B8867
:107E90001B0A4371CB888371CB881B0AC3710820EE
:107EA000704703000120082A14D14A78087812028A
:107EB00002431A80CA788878120202435A804A79AB
:107EC0000879120202439A80CA7988791202024321
:107ED0000020DA80704710B504000120022A05D185
:107EE00000204B780A781B021343238010BDF8B59D
:107EF000060010200F00150003F0DEFB0400012037
:107F0000002C0ED0A0230C22290023806780201D86
:107F1000002D07D003F070F92100300003F044FA7F
:107F20000020F8BD03F080F9F6E7F7B51E000090D9
:107F300008AB142017001D78019103F0BDFB041E4F
:107F400012D0A2230370019B47704380099B0571E7
:107F500046710C220830002B07D0190003F04CF9B1
:107F60002100009803F020FAF7BD099903F05CF9AD
:107F7000F6E737B5041E0FD04388002B0CD0002540
:107F8000C1881323007A172201950095FFF7CDFFD2
:107F9000FF2365806372257037BD000010B50C4962
:107FA00004004A88002A09D08B89002B05D00020C4
:107FB000CB8A0222834201D010BD012213000A2085
:107FC000434300204032C854C81842800472F3E78B
:107FD000225FFF1F0023438003707047094B00217D
:107FE0001A0010B55C88002C06D01C79844203D19D
:107FF0000A234B43D01810BD01310A330329F1D1B4
:108000000020F8E7225FFF1F10B50400407A03F05C
:10801000F3FBFF23637210BD7047043010B580B2CC
:1080200003F0EAF9002803D00421494203F034FBAD
:1080300010BD000070B50025104CA0682580A581FA
:10804000A580A84202D003F06FFAA56000250C4C71
:108050000C4B606D1D80230058331D70A84202D068
:1080600003F062FA656500256068002801D003F01E
:108070005BFA013508340A2DF6D170BDE85FFF1FA9
:108080008C5FFF1FDC5FFF1F70B5041E09D1054D1B
:108090002880A881A880A868002802D003F044FAAC
:1080A000AC6070BDE85FFF1FF0B54B8885B00193F1
:1080B000002343600A7905000F00022A00D07BE00C
:1080C000CA88032A17D98B685E7819783602DC785B
:1080D000D8790E4399781B7A24021B020C43034380
:1080E00053495BBA0B80331D93421ED1042C04D03C
:1080F000631F022B0ED9012015E0019A4D4B12018E
:10810000D35A002B06D00198FFF7BEFF4A4A1369E5
:10811000013313610421B8682E812C80494203F099
:10812000BBFA6860002005B0F0BD434D042C06D0BA
:10813000631F022B0FD9EB680133EB60DBE7019A79
:108140003C4B1201D35A002B05D00198FFF79CFF3E
:108150002B6901332B61374B30000293019B029A4C
:108160001B010193002301998C468B521300634439
:108170009C8003939E81FFF750FF039B041E986031
:1081800016D00421B868494203F086FAFA88010043
:10819000043A200003F030F80199029AFB888A5AC9
:1081A000043B9B18029A8B522B6801332B60A2E789
:1081B000AB690133AB619EE71E4B0293019B1E012D
:1081C000029BF35A002B2DD002998C19A06800282D
:1081D00028D0012A26D1FA889B189BB27352A18914
:1081E000994217D39B1AC018B96803F005F8029B8F
:1081F000A289F35A934200D07DE700222B81A38805
:108200002B80A3686B60029BF2520B4A53680133C8
:10821000536070E7084A9368013393600198FFF751
:1082200033FF68E7044A536901335361F6E7C046F8
:10823000525FFF1FE85FFF1F585FFF1F70B5051EED
:1082400015D10B4C0B4B1880230058331870606D00
:10825000002802D003F068F9656525005035606894
:10826000002801D003F060F90834AC42F7D170BDAA
:108270008C5FFF1FDC5FFF1FF0B51700A12285B0E8
:10828000920001934243394B06001B680C009B1877
:10829000D933FF331D78FDF741FF0430854204DDFB
:1082A0003000FDF73BFF0430C5B2BD4207D33A00B2
:1082B00000213000019B03F067FA05B0F0BD2900F2
:1082C000380003F061F92300C6B250331E700393E7
:1082D000019B29006365380003F03EFACBB202939C
:1082E000002B02D0039B01361E7000262300503362
:1082F00003931B78B34204D8606D002831D100206D
:10830000DBE7029A2800002A04D0013B1000B342A8
:1083100000D02800F700E719387002F0ADFF786050
:1083200000280ED03A78019902F066FF019A3B7856
:108330000136D3180E4A0193D369F6B20133D361E3
:10834000D4E7039B18706065A74205D1084A132043
:10835000D36A0133D362B0E7606803F0E5F808340C
:10836000F2E703F0E1F800236365C8E73409FF1F73
:10837000585FFF1FF7B50D0007000421686803F080
:108380008BF92B89040003702B891B0A43702B88FF
:1083900083702B881B0AC3702E8902250436F6B21F
:1083A000F42E15D81B4B9F4214D10C2003F084F9F6
:1083B0001135011E0CD0902303708E3B0371043BDA
:1083C0004380154B8460C680187802F0EDFF0025CD
:1083D0002800FEBD5C237B43104AD318009358331A
:1083E00001931B78002B0FD1030032003800009955
:1083F000FFF742FF019B05001B78002BE8D13800F6
:10840000009902F0E9FFE3E7054A0725536A0133C3
:108410005362DDE7FEFF0000505FFF1F8C5FFF1F10
:10842000585FFF1FF0B587B0009017200F001600AF
:108430000193FFF7F2FD1325041E19D00C98031EBB
:1084400002D00199201D9847030AE370052302AA70
:10845000A0700430908127700098667003A9938003
:108460000494FFF787FF051E02D0200003F05CF89C
:10847000280007B0F0BD0000F0B587B01F000CABBE
:108480001B780391059301210DAB06001C78049223
:1084900000F0D6F81425002821D02000FFF77EFD3B
:1084A0000135041E1BD01149059B0A780370013267
:1084B000D2B2131EC68001D101231A000B702271A3
:1084C0003000049B03990097FFF7ACFF051E09D10C
:1084D000230021000648074A093302F095FF2800CF
:1084E00007B0F0BD002363802370F8E7545FFF1FDF
:1084F000737F001130750000F8B505000E00064CC2
:10850000064F2368002B02D031002800984704341E
:10851000BC42F6D1F8BDC046F85FFF1F0C60FF1FDC
:108520000123064A5B425380002313715362044ABD
:10853000136053609360D360136170470C60FF1F3A
:10854000F85FFF1F0200002310B506499C00085980
:10855000002801D1625010BD0133052BF6D1132044
:10856000F9E7C046F85FFF1F034A5388181A4342D1
:1085700058414042104070470C60FF1FF0B585B075
:1085800002930AAB1F780CAB1B88009008000E000A
:1085900001920393FFF7E8FF05001120002D1BD186
:1085A0000E48FFF7E1FF04001520002C14D006222E
:1085B0000B99A771E01D02F01FFE019B3000237193
:1085C000029B29006371009B66802370039B656298
:1085D000E381FFF791FF280005B0F0BDFFFF000029
:1085E00010B5FFF7C1FF04000220002C12D06088F4
:1085F0000121FFF781FF606A002801D003F054F8E1
:1086000028220021200002F00FFE012300205B42FF
:108610006380207110BD000030B5074A074C5588B3
:10862000010013780020A54204D05B1A59424B4147
:108630005842104030BDC0460C60FF1FFFFF0000D5
:10864000084A10B501230C00904208D0FFF78CFFB8
:10865000031E04D0037923405A1E9341DBB2180055
:1086600010BDC046FEFF0000024B1879431E984122
:10867000C0B270470C60FF1F70B504000D001600FB
:10868000FFF772FF002804D10D4B9C4200D014303C
:1086900070BD416A03790520002907D012221A40D3
:1086A000102A02D10520002EF2D10F20DB06EFD5D3
:1086B000897E0C20A9428941494249420840E7E7A6
:1086C000FEFF0000030010B5002800D110BD0348D4
:1086D000034A41889142F9D09847F7E70C60FF1FA1
:1086E000FFFF0000002330B5C45CCD5C6C40D45467
:1086F0000133102BF8D130BD0F23002210B5C45C1C
:1087000064002243CA54C25CD209013BF7D210BDB7
:108710000200010010B52032103102F0D5FE10BD6C
:10872000F0B58BB00390102005931700049102F070
:108730008BFF0090102002F087FF009B1324019014
:10874000002B05D000280CD11324009802F0ACFFB8
:10875000019B002B02D0180002F0A6FF20000BB0F6
:10876000F0BD102002F070FF0600102002F06CFF38
:1087700013240500002E00D1AEE0002819D01022ED
:10878000002102F051FD32002900039802F09CFE06
:10879000041E0ED133787F2B51D830000099FFF79B
:1087A000ABFF009B1B787F2B53D801990098FFF7F4
:1087B000A3FF300002F078FF002D02D0280002F065
:1087C00073FF002CC1D1102002F03EFF06001020E4
:1087D00002F03AFF0290002E7CD0002878D03A00B8
:1087E0000F3223000125121105D00F333B4015B283
:1087F0005A4253411BB26A1E1201002B33D0049B14
:10880000D2B298180099029AFFF76CFF013D10222E
:108810000021300002F008FDADB2049F2D017D194A
:10882000AF4242D0002C33D0300002F03DFF029B1B
:10883000002B00D189E7180002F036FF85E72900F8
:108840003000FFF759FF28002549009AFFF74AFF3B
:10885000A7E729000098FFF74FFF28002049019A59
:10886000FFF740FFA5E70F210F4004998A18D9B2FE
:108870008F4208D9D15C06A819540133102BF6D1C8
:10888000029A0199C0E7791A48424141C901F2E7C9
:108890003900300006AAFFF725FF3200039806A929
:1088A00002F012FE10370400BAE7002CBCD13000F1
:1088B000029906AAFFF716FF320006A9039802F0F4
:1088C00003FE082204003100059802F095FCABE796
:1088D0001324A9E71324AAE7002800D06EE733E7A2
:1088E00018BA0011F0B58BB00F00160002250090E9
:1088F00000283FD0002A3DD00B1DDBB218000293A8
:1089000002F0A2FE1135041E34D0FDF747FD05002C
:108910003A000099201D02F027FFEBB20393E370A9
:108920002B0CDBB22F0A00936370FFB22B0E237067
:10893000A7700193FDF72CFD1022010006A802F09C
:1089400013FF2100029A04AB06A8FFF7E9FE051EFB
:108950000DD1039B08223370009B04A9B370019BC7
:108960007770F370301D02F0FFFEFDF71DFD200053
:1089700002F09AFE28000BB0F0BDF0B58FB00D00EC
:10898000149E039004920593002A03D10224200030
:108990000FB0F0BD002EF9D00398FFF7E5FD1424C9
:1089A000071EF4D07278337812021A43B3781B048E
:1089B0001343F27812061A43036A0192934201D3D9
:1089C0000133E3D1002D03D03B7901249B07DED591
:1089D0000822002106A802F027FC059B132404337B
:1089E000DBB21800029302F02FFE051ECFD0059ACD
:1089F0000499043002F0B8FE04223100280002F08D
:108A0000B3FE3900102210310AA802F0ADFE290091
:108A1000029A06AB0AA8FFF783FE041E0FD10822B4
:108A200006A908A802F0A0FE0822311D08A802F03D
:108A30003BFD012807D101990398FDF7C9FC2800E7
:108A400002F032FEA3E70124F9E7000070B51C4CE8
:108A500005002368181E10D0002D14D11A78002AA2
:108A60000CD1981C083202F0C7FB02F0C5FD01359D
:108A7000002808D123681D70012070BD0A3318003A
:108A8000082202F0B9FB2368002BF5D0122002F077
:108A900013FE061E0DD0C1232168037045700231FC
:108AA0001022023002F0A8FB23683100587802F04F
:108AB0007BFC206802F0F8FD00232360DCE7C04661
:108AC0003460FF1FF8B504002020FDF755FB0D4E64
:108AD000A700BB590500002B0DD000280BD0D8787B
:108AE000FF2809D108492A000C55F35907480333D8
:108AF000611802F089FCF8BD290002F0EDFC0028A5
:108B0000F0D1F8E75060FF1F3860FF1F1D9D001176
:108B100070B5064D84006359002B05D0D87802F05B
:108B20006BFEFF226359DA7070BDC0465060FF1FB4
:108B300070B506008CB00C0015000021302268468C
:108B400002F072FB31001022684602F00DFE1D207B
:108B500021000322684402F007FE6846FFF7D8FDB3
:108B60002D21040003222800694402F0FDFD2000AD
:108B70000CB070BDF0B50700160097B001931CABA8
:108B80001D7830221EAB00910AA800211C7802F04B
:108B90004BFB102239000AA802F0E6FD102200214A
:108BA00002A802F041FB0722310002A802F0DCFD1E
:108BB000072202AB9818631E9C41019902F0D4FD74
:108BC00002AB9C732B005A1E934102AAD37300215F
:108BD000102206A802F028FB06221D9907A802F021
:108BE000C3FD1A2002ABC01806221F9902F0BCFD7B
:108BF000102200990EA802F0B7FD102202AB0EA9B8
:108C000008781C78013A6040D2B208700133013113
:108C1000002AF5D10AA8FFF77BFD102212A9040053
:108C20000EA802F0E9FA102206AB0EA908781D780A
:108C3000013A6840D2B2087001330131002AF5D1FF
:108C40000AA8FFF765FD044310222098E4B212A998
:108C500002F08AFD200017B0F0BD70B50E001400C0
:108C60008CB00100102268461D0002F07DFD31002D
:108C7000082204A802F078FD2100082206A802F0CC
:108C800073FD6846FFF744FD04001022280008A980
:108C900002F06AFD20000CB070BDF8B506000D00B2
:108CA00000243719AC4200D3F8BD02F025FC030ABA
:108CB0003B70631CDBB201379D4203D90234F05490
:108CC000E4B2EEE71C00EDE773B506000C000225E8
:108CD000002819D0002917D0032101A8FFF7DDFFD4
:108CE0006B469A793F231A40013313436A4630009A
:108CF000937101A92200FFF71BFF051E04D1032277
:108D0000E01C01A902F078FA280076BD0378580724
:108D1000DA08C00FD20080009B0710439B0F184356
:108D2000C0B2704707230B40C908C9000B4303704A
:108D30007047000070B50400FFF7EAFE134DA40071
:108D40006359002B21D0186A002801D002F0ACFC36
:108D50002B59986E002801D002F0A6FC2B59D86E32
:108D6000002801D002F0A0FC2B59186F002801D078
:108D700002F09AFC2B59586F002801D002F094FCA5
:108D8000285902F091FC00232B5170BD5060FF1F49
:108D90000E4B8000C35870B50C00002B0FD09D689F
:108DA000002D0CD02B78201D0B706B784B70A97C9C
:108DB000FFF7B8FF2B7E23726B69E36070BD102252
:108DC0000021200002F030FAF8E7C0465060FF1F93
:108DD000014B18607047C0464C60FF1F074A0300F4
:108DE0008000825810B5002A06D0D088984203D15E
:108DF000012901D1FFF79EFF10BDC0465060FF1F43
:108E0000F0B5264E95B087000B93BB59050009912C
:108E100012200A92002B31D0D888FFF7A5FB04005E
:108E20001420002C2AD0280010A9FFF7B1FFBB594D
:108E30001E781D6A002E23D00895FDF7EFFA070073
:108E40000020FDF7F1FA0790A379E61D069310AD17
:108E50000CA9089800F0E2FA0EA9280000F0D7FA51
:108E60000B9B0A990493069B09980293079B039610
:108E7000019300970EAB0CAAFFF77CFE15B0F0BD76
:108E8000FDF7CCFA06903000FDF7CEFAE31DA77986
:108E9000079310AB06000893DAE7C0465060FF1F47
:108EA00030B50C4C85002A59030085B00120002AFA
:108EB0000ED018006946FFF76BFF2B591A78D88837
:108EC000054B002A00D1054B6A46072100F0D9FB6B
:108ED00005B030BD5060FF1F0F9400111D940011AC
:108EE00030B5094C8500295985B0102268462531D6
:108EF00002F082F92A591121044BD0886A4600F009
:108F0000C0FB05B030BDC0465060FF1FB9940011D2
:108F100030B5094C8500295985B010226846353195
:108F200002F06AF92A591121044BD0886A4600F0F0
:108F3000A8FB05B030BDC0465060FF1FF79400117C
:108F4000F7B54D4F86001020F4590D0002F07CFB60
:108F5000F3592062186A132200286CD0033A2900C2
:108F60009C6802F049F9F3591A780192002A58D105
:108F70001E6A227D317B944651400122019F11429D
:108F800001D167461740217D914339432175377BD5
:108F90004F40BC4660460027800701D44F08174069
:108FA000012102208F40227D82433A432275377B84
:108FB0005740BC4660460027400701D497080F4041
:108FC0000420227DBF0082433A432275627D002740
:108FD00094466046727B42400A4201D167460F4088
:108FE0000121627D8A433A436275777B5740BC46D4
:108FF00060460027800701D457080F400220627D99
:109000007F00824317436775767B00227E40760798
:1090100001D4BA080A400426617D9200B1430A4394
:1090200062756A78002A08D06278002A05D0052285
:109030000533DA7700221000FEBD0422297911429F
:1090400005D1A17C114202D10533033AF1E7019A1F
:1090500021782C78002A02D10A002100140018225D
:109060000429E8D8042CE6D805206043034A0533D8
:109070001218525CDDE7C0465060FF1F28BA00118D
:1090800010B50A001121024B00F0FBFA10BDC046DA
:10909000539500110B0030B587B001AD2B806B46A6
:1090A00004001100981D082202F0A6F82A000B21E6
:1090B0002000024B00F0E5FA07B030BD7B950011AF
:1090C00010B50A001121024B00F0DBFA10BDC046BA
:1090D000CF95001113B50B0011006A4613706B4653
:1090E00004000622581C02F087F86A460821200076
:1090F000014B00F0C6FA13BDEF95001110B50A0040
:109100001121024B00F0BDFA10BDC0463F96001180
:109110007FB505000B4BAA00D4580800002C0FD0D7
:10912000666F237FE28821780396266F0296E66EAB
:109130000196A46E0094FDF709FC2800FFF7FAFDE4
:109140007FBDC0465060FF1F10B51721FFF7E0FF3D
:1091500010BD000070B50A000D00064B022104008E
:1091600000F08FFA060029782000FFF7D1FF3000C9
:1091700070BDC0461F95001170B586B000236A46C9
:109180001370836804001D78681E0A2859D801A945
:1091900002F082F9060633373B3F43474B4F5300FB
:1091A000180000F042F9062312284BD000281BD1EA
:1091B0006088FFF7D9F90823002813D04279002AE4
:1091C00047D1264B1A78072312070BD5244B1A6870
:1091D0000723002A06D01668002E03D0290001AA12
:1091E000B04703006A4613706B461B786088002BFB
:1091F0002AD1FFF767FC06B070BD180000F06CF9CB
:10920000D4E7180000F087F9D0E7180000F093F9D0
:10921000CCE7180000F0ADF9C8E7180000F0C3F97A
:10922000C4E7180000F0F6F9C0E7180000F0F6F9FE
:10923000BCE7180000F013FAB8E7180000F013FAC2
:10924000B4E707236A46137069466088FFF782FF18
:10925000D1E70523012AC5D1024BB8E7DD5EFF1F28
:109260004860FF1F4C60FF1FF8B52C4F8600F35974
:1092700004000D00002B40D0DA8882423DD15A789C
:10928000062A33D11A78002A2ED0012099681A6A4A
:10929000097D014206D0157B054203D007225A7092
:1092A0000120F8BD0220014204D0157B054201D007
:1092B0000922F4E70420014204D0127B024201D0CB
:1092C0000B22ECE7164B1B68002BE9D05B68002BE8
:1092D000E6D020009847BB5900215B78122BDFD1E4
:1092E0002000FFF715FFDBE70E4BECE7112A04D156
:1092F000002900D032252900F2E7002D08D12000F6
:10930000FFF732F9002803D01023027913430371C9
:1093100021002800FDF798FAC2E7C0465060FF1F01
:109320004860FF1F4C60FF1F70B50E4E8500AB59A3
:109330000400002B13D01B78002B11D10A4B1B68A3
:10934000002B04D05B68002B01D020009847735994
:109350005B78122B03D100212000FFF7D9FE70BDEE
:10936000024BECE75060FF1F4C60FF1F4860FF1F7F
:10937000094B8000C3581020002B0CD01A6A002A19
:1093800009D09B68002B06D0127A1B7E101C9A42D3
:1093900000D9181CC0B270475060FF1F70B50300A1
:1093A0000D0014000220002A30D000292ED01370A6
:1093B0000B78081D53704B789370FFF7A7FCE07093
:1093C000012002212B7A23716B7B034063716A7B3E
:1093D0000A401343042263716E7B1640334363716A
:1093E0006E7BF608F600334363712B7B0340A37159
:1093F000287B014000200B43A371297B0A401343C3
:10940000A3712A7BD208D2001343A37170BD10B59B
:109410000A0001000120FFF7C1FF10BD10B50A00CE
:1094200001000220FFF7BAFF10BD70B506000C0066
:109430000220002E30D000292ED07378201D0B7012
:10944000B3784B70F178FFF76DFC01223579257206
:1094500071794B100800134093401040034388106B
:1094600010408000C9080343C9000B436373B179FE
:109470004B100800134093401040034388100240F3
:109480009200C9081343C9000B4321202373FCF742
:1094900073FE854201D2122070BD2220257AFCF78E
:1094A0006BFE8542F7D823781820042BF4D8637814
:1094B000012BF1D80020EFE7030010B502200029AE
:1094C00009D0002B07D00322481C0A7019000D3266
:1094D00001F092FE002010BD03000222080010B52A
:1094E000002B06D0002904D00E32591C01F084FE56
:1094F0000022100010BD030010B50220002909D081
:10950000002B07D00422481C0A7019000C3201F00D
:1095100073FE002010BD10B5FFF7DEFF10BD030085
:109520000220002906D0002B04D0052200200A705A
:109530001B784B70704703000220002B08D00029D5
:1095400006D05B7800200B70013B082B00D9183047
:109550007047030010B50220002909D0002B07D066
:109560000622481C0A7019000A3201F045FE00204C
:1095700010BD10B5FFF7B0FF10BD02000B000220B8
:1095800010B500290ED0002A0CD0072119701188BF
:1095900059701188090A997011180822D81C01F015
:1095A0002BFE002010BD03000A00022010B5002B86
:1095B0000CD000290AD0997858780902014311800B
:1095C000901CD91C082201F017FE002010BD0300DA
:1095D00010B50220002909D0002B07D00822481C12
:1095E0000A701900921801F007FE002010BD020059
:1095F0000B00022010B500290BD0002A09D0092148
:109600001970117818185970511C062201F0F4FDD8
:10961000002010BD10B5FFF75FFF10BD02000B006A
:10962000022010B5002A09D0002907D051781970FE
:1096300011180622581C01F0DFFD002010BD0300A8
:1096400010B50220002909D0002B07D00A22481C9F
:109650000A701900063201F0CFFD002010BD10B5D0
:10966000FFF73AFF10BD02000B00022010B5002AE0
:1096700006D0002904D018005178FFF753FB0020D2
:1096800010BDF0B585B017001E006A460623050020
:10969000080091819380FEF7C0FC1324011E029004
:1096A0000CD03800B047041E05D1280001A9FEF7F0
:1096B0006FFA041E02D0029801F036FF2800FFF76F
:1096C00001FA200005B0F0BDF0B504008BB00191A7
:1096D00015000021102202A801F0A6FD334EA700BC
:1096E000B85900283CD0C388A34239D10378002B55
:1096F00036D14278062A18D10200010055323531A0
:109700000C3006ABFFF7A9FA002829D12000FFF79B
:109710002FFE020006A902A801F06EFD200002A99A
:1097200002F012F801200BB0F0BD816E002917D0B5
:109730000B8A112A28D19D420ED101981231093A83
:1097400001F0B2FE012807D1BB5920009D6EFFF742
:109750000FFE29000200DEE732212000FFF7D8FCCF
:109760002000FEF701FF061E1BD0416A002918D019
:109770000B8AAB4215D108220198123101F094FEF8
:1097800001280ED1716A0AE09D42E9D108220198B0
:10979000123101F089FE0128E2D1BB59996E8A7E0F
:1097A000B9E7200001F060FEBCE7C0465060FF1F33
:1097B000F0B56B4D87007E5985B0337802900393E6
:1097C000002B00D087E0B368346A019370780628D4
:1097D00017D101221B7D134202D0217B114218D1E7
:1097E0000222134202D0217B114251D104221342A2
:1097F00003D0237B134200D08BE0019B5A7DEB59B1
:1098000091E007380428F8D801F046FE032E42679D
:109810008300B36E002B03D11C2001F015FFB0664E
:10982000EB599C6E002C1CD010220021200001F06E
:10983000FBFC0298FFF79CFD01002000FFF72DFACA
:1098400001F05AFE2082200008211230FFF725FA8D
:109850000298FFF78DFDA076EB592100D888FFF71D
:109860000FFC0822EB591CE0B36E002B05D01A0048
:10987000198AF0881232FFF70DFC0222019B197D34
:10988000EB5911423DD0207B10423AD0073208E01C
:10989000F488FCF7DBFD01002000FFF711FC0A2231
:1098A000EB595A70029B9C002A595378073B042BB2
:1098B00011D8D088FEF758FE00284ED0C3895A0828
:1098C000D2182849029B0298CB542B5941180433D3
:1098D000254801F099FD05B0F0BDFCF79FFD0300A0
:1098E0000120834201D100200393EB59DE88FCF76D
:1098F0009BFD039902003000FFF7ECFB019AEB5946
:10990000117D042211420CD0217B114209D00B227F
:10991000C7E7F688FCF73CFD01003000FFF7EEFBDF
:109920006BE7019A527D01210A4204D0607B084214
:1099300001D00C22B5E702210A4204D0607B084224
:1099400001D00E22ADE704210A4204D0627B0A4214
:1099500001D01022A5E71222A3E7FA225200B0E7B5
:109960005060FF1F5460FF1F279D001110B5064B6C
:109970001A780423100018401A4200D00348FFF759
:1099800027FA002010BDC046DD5EFF1FA43DFF1F6B
:1099900070B50400FFF7D4FA051E43D12000FFF78D
:1099A0007FFA234EA400A0598268937CDB0708D578
:1099B0000321036A1B790B40012B02D1017F0B436A
:1099C0000377431DD97F8B1E022B0DD8022900D0AF
:1099D0000121C088FCF790FF042133591A7F597088
:1099E0000A431A77280070BD01290CD102231022E6
:1099F000437000210C3001F017FC30591021353034
:109A0000FFF74BF9EEE70529ECD10223D11843709B
:109A100010220C3001F0F0FB04233259117F0B436C
:109A20001377EAE708251828DCD1053DDAE7C046B8
:109A30005060FF1FF0B58BB0059143887E4F9E00AC
:109A4000F45915000493002C15D1012902D00020EF
:109A50000BB0F0BD101D57781678FFF757F9EB687B
:109A6000320002932B7A0499019300903B0020006E
:109A7000FCF70CFFEBE7E388049A934201D008203F
:109A8000E6E72378012B00D1D4E0059B581E092876
:109A900000D9CFE001F000FD05CE0A29CC506C853D
:109AA0009AB229000498FFF773FFD1E7200029003C
:109AB0001022453001F0A0FBB9594B78042B02D19C
:109AC000013B4B70C3E70B000A00253335320C31E4
:109AD0000498FFF795F90498FFF702FA0522431E50
:109AE0009841BB59C0005A70B2E7200029001022EB
:109AF000553001F081FB049B4F4C9D00295904987F
:109B00000A0006AB55320C31FFF77AF929591022B9
:109B1000453106A801F0C8FC012808D10498FFF7D8
:109B2000F7F90590002804D106222B595A700598A0
:109B30008EE708230593FAE763780C2B7AD1E36E5E
:109B4000002B03D11C2001F07FFDE066BB59D86ECD
:109B500000286FD01022290001F04EFBBB59049859
:109B6000DC6EFFF705FC0D22A076BB595A706EE73C
:109B7000E06E00285ED063780D2B5BD12B88082225
:109B80000382A91C123001F037FBBB599A68517D42
:109B90000222114226D0186A407B104222D00C3299
:109BA000E4E763780E2B45D1236F002B03D11620F9
:109BB00001F04AFD2067BB59186F002803D010221E
:109BC000290001F019FB0F22BB59CFE763780F2B57
:109BD00030D1206F0622691C103001F00DFBBB59FB
:109BE0009A68517D0422114203D0196A497B1142BF
:109BF000D5D100210498FFF78BFA28E7636F002B7B
:109C00000DD0BB59586F0028F3D01022290001F065
:109C1000F3FA0122BB5952425B6F1A61E9E7142043
:109C200001F012FDBB5960675B6F002BE9D126E79D
:109C30002978DFE707200BE75060FF1F10B5064CBF
:109C4000207001F021FD06212078FDF791FF0348E7
:109C5000FEF778FC10BDC0466360FF1FDD8D00116C
:109C600000200BB270B50D00834216DA264B18782F
:109C700001F0DAFC041E0DD00378922B0ED0A02B3D
:109C800037D0224B1878FF283AD0210001F08CFB06
:109C9000002835D180200002684070BD43780E2B2B
:109CA0000BD03E2BEDD18378052B12D0082BE8D1B9
:109CB00081798088FFF7D8FA08E0154B82889A42AC
:109CC000DFD183681878591CFEF7C0FE002817D131
:109CD000D7E7104B1B785B0712D50F4B1B68002B87
:109CE0000ED09B68002B0BD0C289811D80889847BD
:109CF000ECE7FFF741FAA068002801D001F014FC5E
:109D0000200001F0F1FCC5E76360FF1F9D3DFF1FD0
:109D100018200000DD5EFF1F4C60FF1F10B50078AB
:109D2000FFF712FA10BD10B50078FFF7FDFA10BD6D
:109D30000C234343084A10B59B185A68002A03D0E5
:109D4000012901D1904710BD9B68002BFBD0002951
:109D5000F9D19847F7E7C0468060FF1F0123834091
:109D6000094A10B5946B1C439463506B984350633D
:109D7000D46B20009843012901D120001843D063FF
:109D8000116B0B43136310BD00800040F0B500243D
:109D90000127154B85B0DA6B144E03921A6C0192B1
:109DA000DA64019BE3403B4217D0039DE5403D4010
:109DB0000295E5B202992800FFF7BAFF316A736A8B
:109DC000002908D03900002B01D0029979402800E1
:109DD000FFF7C4FF01E0002BF9D101340C36172C3A
:109DE000DFD105B0F0BDC046008000406460FF1FB9
:109DF000064B01215A68C2400A4204D01B68C34086
:109E00001800084070471B6DF9E7C046008000400D
:109E10000122064B8240002903D0D9680A43DA6048
:109E20007047D9689143D960FAE7C04600380040CE
:109E300030B5032444430F4BE25C1B199C785D78DA
:109E400001232D1B0135AB40013BA340A140DB4367
:109E50000C00122807D808499200521811681940BE
:109E60002143116030BD054A11680B402343136044
:109E7000F8E7C0466FBA001108F0004014F0004047
:109E8000C21F70B5D4B20623092C0BD80125084C8B
:109E90009540002908D00021FFF7CAFF23682B4313
:109EA00023600023180070BD2368AB43F8E7C04669
:109EB00000380040214BF0B51B185B78022B21D1F4
:109EC000032444431E4A1F4EA35C121994780122B6
:109ED00015008540B76B013CE4B23D43A240B56339
:109EE000194C122815D89B0000290CD117495B1872
:109EF00099680A439A600123205C154A83401168DF
:109F00000B431360F0BD11495B1899689143996048
:109F1000F1E70E4B00290DD159690A435A61225CC1
:109F20001328E8D00123203A93400A4908680343E4
:109F30000B60E7E7596991435961F0E76460FF1FDF
:109F40006FBA001100800040B4BA001100F0004068
:109F5000A0F00040A4F00040F8B500241B4E1C4DBA
:109F60001C4B1B5D012B1FD1194A9269E2401A421A
:109F70000BD00122B25693402200143AD2B2022AE8
:109F800009D815494A6913434B61013402360C352F
:109F9000172CE5D1F8BD0022B2560F499200521895
:109FA00091680B439360F0E7022BEED1E7B23800E3
:109FB000FFF71EFF01235840C1B23800FFF77AFFB8
:109FC0003800FFF715FF6877DFE7C04641BA001198
:109FD0006460FF1F6560FF1F00F00040012202382F
:109FE0008240054B002903D059690A435A617047E2
:109FF000596991435961FAE700380040F8B50E00FD
:10A0000001210F008740114A0400D368FD43BB4380
:10A01000D360831E8B4201D8FFF7E0FF00212000B0
:10A02000FFF72EFF0A4A0B4B5168012E05D1394329
:10A030001B1951605E700020F8BD2940516002225A
:10A040001C1962709A6915409D61F4E70038004060
:10A05000008000406460FF1F012210B58240074B62
:10A06000002906D019680A431A600121FFF7C6FFCC
:10A0700010BD196891431960F7E7C04600800040A1
:10A080000C2370B5002543430A4A29009B181D7014
:10A09000094B04001B185D70FFF7B0FF0123A340BC
:10A0A000064928000A681A430A6005490A689A4363
:10A0B0000A6070BD8060FF1F6460FF1F3480004035
:10A0C0003080004070B504000E00FF2813D0032537
:10A0D0000540FFF7D5FF084AA3089B009B183F22C5
:10A0E000ED00AA40AE401968200091433143196049
:10A0F0000121FFF78DFE70BD18380040F8B50C2423
:10A100004443134B0500E4186368002B03D1A36894
:10A110001220002B1AD0022201270E4B00215B19BE
:10A120005A7028002770FFF769FF63681E1E08D069
:10A13000A3683E00002B04D02800FFF759FE4640DC
:10A14000F6B228003100FFF709FE0020F8BDC04636
:10A150008060FF1F6460FF1FF7B5C420FF222B4BF8
:10A1600080001958002491433F3A0A431A50802234
:10A17000274F5202274E1A60274B1D5D002D21D01C
:10A18000A31E012B03D80121E0B2FFF727FF012D09
:10A1900018D11F4B9B69E3402B4213D0E3B2180048
:10A1A0000193FFF725FE01000198FFF755FFE3B289
:10A1B000143B022B1DD801217156184A8D4053695A
:10A1C000AB4353613B7F002B0DD0E5B22800FFF776
:10A1D00095FF2800FFF70CFE7B7F0100834202D031
:10A1E0002800FFF7A5FD01340C370236172CC3D128
:10A1F000F7BD012100237156F3568D40074A9B009D
:10A200009B189A68AA439A60DCE7C04600E100E028
:10A210006460FF1F41BA00116560FF1F00F000403D
:10A2200010B501210400FFF7E9FE0123044A0020D4
:10A2300011194B70A34091690B43936110BDC04647
:10A240006460FF1F70B50E0015000400FFF718FFD3
:10A250000C236343094A20009B189D605E60FFF752
:10A260004DFFF021064B074A8900051E5A5002D0C7
:10A270002000FFF705FF280070BDC0468060FF1F6B
:10A280000000FF1F8D9D001170B5134D07202C7825
:10A29000002C1FD1982221005200280001F044F820
:10A2A0000123C420FF222B700C4B80001C635C63D5
:10A2B0000B4B1C605C600B4B195891433F3A0A43AF
:10A2C0001A50802252021A600D20074A074900F0F6
:10A2D000DBFF200070BDC0466460FF1F00800040AF
:10A2E000A0F0004000E100E059A10011599F0011C9
:10A2F00070B51D0002240C2910D8094ACA40D207A3
:10A300000CD5FBF745FF041E08D1059A04992800D7
:10A31000FBF75AFFFCF7C8FDFFF728FB200070BDD4
:10A320001210000030B50D7802232C009C43184217
:10A3300001D02B431C0008252300AB43284201D049
:10A340002B00234320241D00A543204201D01C43A1
:10A3500025002A230D70184204D011781E3B0B43B0
:10A36000137030BD0028FCD10C2113788B43F7E724
:10A37000F8B51D0006AB1B88140007AA0E000B20C1
:10A380001778002B27D10A78022A49D14A685078D9
:10A3900011780002244A08438018042840D801F0AC
:10A3A0007BF803121D1B2300F06800F0E5FF021C80
:10A3B000C0B2B84200D93A1CD2B22000F1682A805B
:10A3C00000F01AFF06E00222F3681B882A8023703F
:10A3D0001B0A63700020F8BD0622EEE701232B80E4
:10A3E000F3681B782370F5E7F368002B16D008227A
:10A3F0002A801A8822701A88120A62705A88A270FB
:10A400005A88120AE2709A8822719A88120A627136
:10A41000DA88A271DB881B0AE371DBE72B80D9E7BE
:10A4200001202B80D7E7C04600D6FFFFF7B5160006
:10A430000A781D0008AB1F880C000123022A18D1DE
:10A440004A685078117800022B4A08438018032884
:10A450000FD801F021F802254439E06800F08CFFA4
:10A46000C0B20723B84204D37B190193152B02DD38
:10A470000D231800FEBDE0682A003100C01900F06D
:10A48000BBFE6B4600209B88E268D0541B4B1B68C8
:10A49000834203D01B68834200D098470023E8E73B
:10A4A0000B23002FE5D1022DE2D1737832781B0205
:10A4B0001343E2681380114B1B68002BEED01B681E
:10A4C000002BEBD00120E8E70B23002FD1D1062D84
:10A4D000CED12A003100E06800F08EFEDEE70B23CB
:10A4E000002FC6D1012DC3D132787533012AC0D8CF
:10A4F000E3681A70D2E7C04600D6FFFF7062FF1F04
:10A5000070B50C001500072837D800F0C5FF0414FB
:10A5100036361B36242E182015290BD8184E162235
:10A520000021300000F080FE22002900300000F001
:10A5300063FE002070BD18200229FBD11288114B48
:10A540001A80F6E718200829F4D10A000E482900DD
:10A5500001F012F9EDE718200129EBD10B4B10782F
:10A560000B49DA69FFF7DEFEE3E718200129E1D1A4
:10A57000064B10780749DA6BF4E70220DAE7C046A9
:10A580005862FF1F463EFF1F3C3EFF1FCC3DFF1F92
:10A59000F43DFF1F143EFF1F030010B50020DB0732
:10A5A00004D50721024A034800F08CF810BDC046CC
:10A5B000CCBA0011CC3DFF1F054A030010680028EB
:10A5C00003D082889A4201D1806870470068F6E71C
:10A5D0006864FF1F0A88030008009A4204D08A8832
:10A5E00004309A4200D0002070470000F8B5F222F3
:10A5F00000230D4F0D4E7968050042433370994298
:10A6000000D07B600A4C0021200000F00DFE0023EA
:10A610001A007C60AB4202D100203370F8BD0133D8
:10A620002280DBB2F234F5E76065FF1F5E65FF1F35
:10A630006C64FF1F73B56B460190060068461500F9
:10A640001980FCF763FF041E11D1002D0FD076890D
:10A65000002E11D00C2000F0F7FF00280ED0084A81
:10A660000460136886808560002B02D11060200092
:10A6700076BD1A001B68F7E70224F8E71324F6E713
:10A680006864FF1F012100220A4B10B549420A4CA1
:10A69000198099809A719A70084B20700120198056
:10A6A0005A60FFF7A3FF2078FCF78EFF0448FDF700
:10A6B00049FF10BD7862FF1F6865FF1F6065FF1FBF
:10A6C00071A70011022310B5002802D0FFF7B2FFD6
:10A6D0000300180010BD0000030010B50020DB07C8
:10A6E00004D50421024A0348FFF7A4FF10BDC04669
:10A6F000E0BA00114C3EFF1FF0B50E2687B0039361
:10A700000CAB1F8802ABF61805000800310002925E
:10A71000FDF77EF804000120002C0FD03088FFF7F1
:10A720004BFF03000E20002B08D05E68002E05D0E2
:10A7300021002800039B029A0097B04707B0F0BDA4
:10A740000A4B10B5984207D10122002352420A80D9
:10A750008B708A808B7110BDFFF73CFF0028FAD008
:10A7600001235B42038000238370F4E7FFFF0000B6
:10A77000F8B5050001290AD1134E00243388F227C9
:10A78000AB4219D028001149FFF7DAFF06E0022991
:10A7900004D10139FDF754FF0028EDD0F8BD3B008E
:10A7A00063437268D018D35A002B09D03A000021B5
:10A7B00000F03AFD0134E4B2054B1B78A342EED819
:10A7C00001235B423380DDE76065FF1F7862FF1F76
:10A7D0005E65FF1F10B5FFF7FDFE030000208342FA
:10A7E00000D0987810BD0000F0B589B01C000EAB09
:10A7F00080CB03901E8810AB1B78049202930B7AD7
:10A800000D00DB0616D42B780593022B24D0049878
:10A81000FFF7D2FE002812D003689C46002B0ED012
:10A82000029B2200019329003B0064460398009696
:10A83000A04705E00498FFF7BFFE002802D10E20D4
:10A8400009B0F0BD8368002BF9D00A2229000398D3
:10A8500098470028D7D0F3E76B6858781A786B4B85
:10A86000000210439842D2D8043B984210D2684B61
:10A87000984242D015D8674BC0180128C7D80B2082
:10A88000002EDDD1EB681A7859683A80200028E064
:10A89000614BC018032800D979E000F0FDFD846AFF
:10A8A000789E5E4B9842B2D10B20002EC8D1012376
:10A8B0003B80EB6831001B7823706889013080B2DF
:10A8C000FCF7A6FF3A88031E0ED0017802328A18E0
:10A8D0003A80428962704289120AA27059680278ED
:10A8E000E01C00F089FC06E004323A8031000422CA
:10A8F000601C00F099FC0020A2E70B20002E9FD1E5
:10A90000EB6807A91E8804233B80330A30002670B9
:10A910006370FCF77DFF051E28D004AB9A890E23D7
:10A9200004A95B183E49C668FCF7E6FF00280BD176
:10A930002B783C486A680599FBF79CFB002803D1FB
:10A94000012304AA5B42D3813278022A06D17168BE
:10A95000201D00F051FC3B8802333B800E2304AAEB
:10A960009B181B88A3701B0AE370C4E704ABDE814D
:10A97000F4E70B20002E00D062E7E9680398FFF7A8
:10A9800029FF02233B802070000A6070B3E70B2090
:10A99000002E00D054E70222EB681B883A80237017
:10A9A0001B0A6370A7E7E86800F0E6FCC2B2030088
:10A9B0000720B24200D243E70DD00299DBB27118F2
:10A9C000994202DB921BD3B20293029BE9681A0000
:10A9D0003B8089195AE70023F6E70B20002E00D0B0
:10A9E0002EE70722EB683A801A7822705A78627054
:10A9F0005A88A2705A88120AE2701A792271DA888B
:10AA00006271DB881B0AA37175E7C0460429000048
:10AA10000228000000D8FFFFFFD6FFFF0328000038
:10AA2000FFFF000010BA0011F0B58DB06B4600209A
:10AA3000089120229B5E83423DDAA64B187800F0F5
:10AA4000F3FD071E32D00378B02B2CD100790238E9
:10AA500016281FD800F088FD17001E001E001E00DB
:10AA600031001E0096001E001D011E0052011E0036
:10AA700073011E00CD011E0050021E001E001E00AC
:10AA80008E021E00E302944B94491B8878880B8049
:10AA9000FBF730F83800FCF7B1FF914B1B68002B37
:10AAA00001D038009847380000F01EFE8020089B37
:10AAB0000002434018000DB0F0BDEE22002187488F
:10AAC00000F0B2FB0BAA3B7B7989388900923A00EF
:10AAD0000D32FCF7B5FD0400804B1B78002C3FD1F4
:10AAE00046E0804B788805937F4B4100CB5A0BAEF4
:10AAF000073BDBB232880293002301937B4B21009A
:10AB000006930093059BFFF76FFE744D002810D14C
:10AB1000069B3A8A1B889A420BD13800059912305D
:10AB200000F0C2FC002804D02B7862899B00EB184F
:10AB30005A80162306A81B18328820007989FCF752
:10AB4000DBFE2B7804009A00AA1851880029C3D094
:10AB50000133DBB22B70002807D006A9C98A918087
:10AB6000634A12889A42BCD802E00121494291808E
:10AB7000002B04D059497888FAF7F0FF8AE73E891C
:10AB80000A2479E000253E89574B06937B88069A74
:10AB90005B009B5A033B9D4202DB002DF0D05BE043
:10ABA000162206A812183B7B798900923A003000E1
:10ABB0000D32FCF745FD0590002858D04689017AF2
:10ABC0007888FCF707FD041E44D1464B788807932C
:10ABD000069B4100C95A454B0439C9B206AAD28A1C
:10ABE00006930291019400930599079BFFF7FCFDE2
:10ABF000041E2FD1069B39491A88931C002D26D19B
:10AC00004B807988384B4900CB5A5119033B8B4212
:10AC100020DD059B31485B8941190B71A91C013569
:10AC2000C9B2EDB2059145191B0A2B71059B2D493F
:10AC30000433181800F0E0FA2C4B059A1B88D3183F
:10AC4000DDB22C4B9E4205D00136B6B29CE7498856
:10AC50009942D6D0002D0CD0204C2800618800F0FD
:10AC6000FBFB207021007888FAF788FF12E7059C2B
:10AC7000F0E7002C00D183E77B78142B00D109E7A3
:10AC800016493B794E800B700C717888FAF728FFD3
:10AC900000E7162406ABE41821003889FCF7B8FD5C
:10ACA000011E00D1B7E1788822880F4C45002C5B4B
:10ACB0000A4D013CE4B2029400240F4B019400952C
:10ACC000FFF792FD041E00D014E129007888FAF7FE
:10ACD00065FFDFE66865FF1F3C3DFF1F8062FF1FC9
:10ACE0007462FF1F7463FF1FB05EFF1F6464FF1F69
:10ACF0003A3DFF1FFFFF00008262FF1F162406ABD4
:10AD0000E41821003889FCF783FD011E00D182E19F
:10AD100078882288AE4C45002C5BAE4D013CE4B2F5
:10AD200002947C89AC4B01940095FFF75DFD041EF5
:10AD300000D0DFE029007888FAF73AFFAAE600257C
:10AD4000A44B1D803B00F6331B78A24A78880792FB
:10AD5000AB4208D99E4B12880693069943005B5A72
:10AD6000013B9A4203DB0799FAF72CFF92E616247F
:10AD70006B00FB18059306ABE418059B21001889AE
:10AD8000FCF746FD011E03D1059B01241E8973E7D4
:10AD90007888924B2288069C099343001B5B904E57
:10ADA000013BDBB20293002300960193099BFFF75E
:10ADB0001BFD041E02D0059B1E895DE77B88069A59
:10ADC0005B009B5A079A108832881218934202DC63
:10ADD0001B1A013B33807F4C0230328809990019DD
:10ADE00000F00AFA2388328801359B182380EDB2DF
:10ADF000A8E70BAA3B7B7989388900923A000D328B
:10AE0000FCF71EFC00250590059B002B04D10A24AD
:10AE1000002D00D16EE060E0059B7888197AFCF780
:10AE2000D9FB0100041E63D1694C6C4B78880694F1
:10AE30000993069B4400E45A694B063CE4B20BAE0E
:10AE4000328807930294019100930599099BFFF7BB
:10AE5000CBFC041E4CD1079B5E491B881A1D002D9C
:10AE600030D14A80059B5B4C5A8963191A716B1C5F
:10AE70009BB2E318120A1A71162306A832881B180F
:10AE800079890598FCF738FDFF21AA1C2E1D033592
:10AE90000B00059092B2B6B2ADB2002803D006AB5B
:10AEA000DB8AD9B21B0AA218651911712B714C4D9E
:10AEB000301D2A884949201800F09EF92B88F61881
:10AEC000B5B2A1E74988914207D17A880699520024
:10AED000525AEB18053A9A42C4DC3E4C280061886D
:10AEE00000F052FB207021007888FAF775FED1E55A
:10AEF000002DF2D13E89BFE6162606ABF6183100CA
:10AF00003889FCF785FC3D000400FA3500282DD077
:10AF1000037A9B060CD400227B89398978880092B9
:10AF20003A000C32FFF7E8FB041E10D03E8915E012
:10AF30003088FFF741FB00281AD08368002B17D018
:10AF40002100122278889847041EE4D0EEE72B787F
:10AF5000002B02D17888FAF74FFE00262B78002BC1
:10AF600000D097E5002C00D194E585E60124DDE7CB
:10AF70000E24DBE7162506ABED1829003889FCF70F
:10AF800047FC041E47D0037A9B0611D4154A7B88E0
:10AF90001188994203D01448814207D11380134B82
:10AFA000F2261D780023D9B2A94221D30924A1E7B2
:10AFB0002888FFF701FB00282FD08368002B2CD0B6
:10AFC0002100122278889847041EDFD092E7C046FD
:10AFD000B05EFF1F8062FF1F8262FF1F7463FF1F4E
:10AFE0006464FF1F6065FF1FFFFF00005E65FF1FB9
:10AFF00031005943546801336018615A0029D2D195
:10B000003C0008342100F22200F0F6F82100788894
:10B01000FAF7FAFD3EE501246CE70E246AE71D4BC2
:10B020001A887B889A4231D07888FAF7F7FD31E5A3
:10B03000F223059851684343CD18C95A00291FD0FF
:10B040003B7A012B0BD16C88AB887888AA1D0094C1
:10B05000FFF752FB041E02D000233B722E88F2221F
:10B060000021280000F0E0F800232B80059B01332D
:10B07000DBB20593084B05991B78064A8B42D7D85B
:10B0800001235B421380002CCED0F5E5002634006E
:10B090000596EFE76065FF1F5E65FF1F70B5040052
:10B0A0000E001500FFF796FA031E08D1310005487F
:10B0B000FFF790FA03001120002B02D01C80002023
:10B0C0009D7070BDFFFF0000F8B50B4F06003B7888
:10B0D0000D001400FF2B0ED00A2000F0EDFA011E27
:10B0E00009D0B1230380002346800371C580048109
:10B0F000387800F059F9F8BD8D3EFF1FF7B50F0005
:10B1000008A90600088809A90B240988002821D16C
:10B110000234022B1ED1557813782D021D432B00CB
:10B120008B4301937334002B14D1FB68300019005A
:10B130000093FFF74FFB019C85420BD02A003000A3
:10B140000099FFF7ABFF041E04D12A003000798973
:10B15000FFF7BAFF2000FEBDF0B50E7885B0039072
:10B160000AA805880120022E0DD14C682778647842
:10B1700024023C43054FBC4205D10398DBB2019643
:10B180000095FFF7BBFF05B0F0BDC04602290000E7
:10B19000034B10B51B68002B00D09847FEE7C04654
:10B1A0006C65FF1F07B501A8FFF7F2FF044A0548C9
:10B1B0000021121A00F0B8F8F8F71CFBFEE7C046B1
:10B1C0007065FF1F903EFF1F01B40248844601BC1A
:10B1D000604700BFE130FF1F01B40248844601BC54
:10B1E000604700BFADAE000001B40248844601BC18
:10B1F000604700BF3D18000001B40248844601BC0E
:10B20000604700BFE94C010001B40248844601BC1C
:10B21000604700BF8B52010001B40248844601BC64
:10B22000604700BF9DA9000001B40248844601BCEC
:10B23000604700BF154D010001B40248844601BCBF
:10B24000604700BF2526000001B40248844601BCC7
:10B25000604700BF3935FF1F01B40248844601BC76
:10B26000604700BF6571010001B40248844601BC1B
:10B27000604700BF056A000001B40248844601BC73
:10B28000604700BF017F000001B40248844601BC52
:10B29000604700BF812BFF1F01B40248844601BCF8
:10B2A000604700BFE12AFF1F01B40248844601BC89
:10B2B000604700BF1D4B010001B40248844601BC39
:10B2C000604700BFA533FF1F01B40248844601BC9C
:10B2D000604700BF6D33FF1F01B40248844601BCC4
:10B2E000604700BF4550000001B40248844601BCDD
:10B2F000604700BF392BFF1F01B40248844601BCE0
:10B30000604700BF8D12000001B40248844601BCB2
:10B31000604700BF4D1F000001B40248844601BCD5
:10B32000604700BF212DFF1F01B40248844601BCC5
:10B33000604700BFB70E000001B40248844601BC5C
:10B34000604700BFB14E000001B40248844601BC12
:10B35000604700BF6DBC000001B40248844601BCD8
:10B36000604700BF691F000001B40248844601BC69
:10B37000604700BF0124000001B40248844601BCBC
:10B38000604700BFDD52010001B40248844601BCA1
:10B39000604700BF7918000001B40248844601BC30
:10B3A000604700BFED4A010001B40248844601BC79
:10B3B000604700BF594F010001B40248844601BCF8
:10B3C000604700BF2534FF1F01B40248844601BC1A
:10B3D000604700BF5D17000001B40248844601BC0D
:10B3E000604700BF7D18FF1F01B40248844601BCBE
:10B3F000604700BF6532FF1F01B40248844601BCAC
:10B40000604700BFE928000001B40248844601BC3F
:10B41000604700BFA946010001B40248844601BC50
:10B42000604700BFF94C010001B40248844601BCEA
:10B43000604700BFE117000001B40248844601BC28
:10B44000604700BF5952010001B40248844601BC64
:10B45000604700BFB131FF1F01B40248844601BC00
:10B46000604700BF350E000001B40248844601BCAD
:10B47000604700BF091B000001B40248844601BCBC
:10B48000604700BF0D52010001B40248844601BC70
:10B49000604700BF5522000001B40248844601BC49
:10B4A000604700BF4D36FF1F01B40248844601BC0F
:10B4B000604700BFCD4C010001B40248844601BC86
:10B4C000604700BFE533FF1F01B40248844601BC5A
:10B4D000604700BFE548000001B40248844601BC53
:10B4E000604700BF5147010001B40248844601BCD7
:10B4F000604700BFEDA5000001B40248844601BCCE
:10B50000604700BF2951010001B40248844601BCD4
:10B51000604700BFC521000001B40248844601BC59
:10B52000604700BF2124000001B40248844601BCEA
:10B53000604700BFD949010001B40248844601BCFC
:10B54000604700BFF30E000001B40248844601BC0E
:10B55000604700BF792EFF1F01B40248844601BC3A
:10B56000604700BF5125000001B40248844601BC79
:10B57000604700BF6136FF1F01B40248844601BC2A
:10B58000604700BFA54F010001B40248844601BCDA
:10B59000604700BF090E000001B40248844601BCA8
:10B5A000604700BFBD30FF1F01B40248844601BCA4
:10B5B000604700BFC9A9000001B40248844601BC2D
:10B5C000604700BFB130FF1F01B40248844601BC90
:10B5D000604700BF156B010001B40248844601BCFE
:10B5E000604700BFE528FF1F01B40248844601BC44
:10B5F000604700BF492DFF1F01B40248844601BCCB
:10B60000604700BFD91B000001B40248844601BC5A
:10B61000604700BFB54C010001B40248844601BC3C
:10B62000604700BF2146010001B40248844601BCC6
:10B63000604700BFF54E010001B40248844601BCDA
:10B64000604700BF75A9000001B40248844601BCF0
:10B65000604700BF3D4B010001B40248844601BC75
:10B66000604700BF456B010001B40248844601BC3D
:10B67000604700BFC56D010001B40248844601BCAB
:10B68000604700BF291C000001B40248844601BC89
:10B69000604700BFC926000001B40248844601BCCF
:10B6A000604700BF5549010001B40248844601BC0F
:10B6B000604700BF014C010001B40248844601BC50
:10B6C000604700BF1D4D010001B40248844601BC23
:10B6D000604700BF851F000001B40248844601BCDA
:10B6E000604700BFDD66010001B40248844601BC2A
:10B6F000604700BF434D010001B40248844601BCCD
:10B70000604700BF055E000001B40248844601BCEA
:10B71000604700BF8552010001B40248844601BC65
:10B72000604700BF9134FF1F01B40248844601BC4A
:10B73000604700BF3555000001B40248844601BC93
:10B74000604700BFF92AFF1F01B40248844601BCCC
:10B75000604700BF311B000001B40248844601BCB1
:10B76000604700BF090E000001B40248844601BCD6
:10B77000604700BF4551010001B40248844601BC46
:10B78000604700BF810E000001B40248844601BC3E
:10B79000604700BF5118FF1F01B40248844601BC36
:10B7A000604700BF0D35FF1F01B40248844601BC4D
:10B7B000604700BF5933FF1F01B40248844601BCF3
:10B7C000604700BFC94A010001B40248844601BC79
:10B7D000604700BFB352010001B40248844601BC77
:10B7E000604700BF3936FF1F01B40248844601BCE0
:10B7F000604700BFC51D000001B40248844601BC7B
:08B80000604700BF1147010081
:10B808000001010302030303040305020602070201
:10B81800080209000A030B030C020D000E030F03B4
:10B82800100311031303140315001600C13B001184
:10B83800F53B001100000000020000004AB80011AA
:10B84800192A0F180A000000F1590000FD24000011
:10B85800414601004D7C0011619C0011B57000113A
:10B86800517A00116152001129AA0011D54E001118
:10B87800B53D0011E53E001100000000161600005D
:10B888000200000094B80011F4FFF3FFD2FC00009E
:10B898002540001100000000000000005475796187
:10B8A8000042312E340030303134006769746875D5
:10B8B800622E636F6D2F707676780042544830316F
:10B8C8000000000002000000E0B80011292A282A20
:10B8D800272A262A252A242A0A180000E20400001A
:10B8E8007102000078EC000074400000102700008E
:10B8F80060F0000006640000204E00000000000018
:10B90800050000001F501D00023CB4000001140097
:10B9180014000000810200003031323334353637EC
:10B92800383941424344454600000000655600113D
:10B93800B956001100000000020000004CB90011C7
:10B948006F2A6E2A1A18000001A0000000000000EB
:10B958006410B71DC8206E3BAC30D9269041DC7608
:10B96800F4516B6B5861B24D3C7105502083B8EDB2
:10B9780044930FF0E8A3D6D68CB361CBB0C2649BD6
:10B98800D4D2D38678E20AA01CF2BDBDFB349B5FFB
:10B99800800000800010000000000000B75C00116B
:10B9A80041730011DB5C0011497700115F5D0011E4
:10B9B8001F770011D55D0011F5760011275E001183
:10B9C800BD7800118F5E0011BD780011C15E0011B5
:10B9D80077780011D55D0011AD7600114D5E00112C
:10B9E800557800110000000000000000335F0011CE
:10B9F80055780011955F001159730011052A042A22
:10BA0800012A002A02290328012800280118001801
:10BA18000000000000000000000000000000008797
:10BA280001010201020101020102030304010301F1
:10BA3800010101010303020103000D000E001000C3
:10BA4800110013001401070108010A010B011C0170
:10BA58001D02040205020702080219021A021C024A
:10BA68001D03010302031700020100050400080773
:10BA7800000B0A001716001D1C0102010105040134
:10BA88000E0D011110011413011716011A190202E3
:10BA980001020B0A020E0D021110021413021716EE
:10BAA800030504030807030B0A030E0D0001020334
:10BAB80007090A0B0E0F101112141718191A1B1F59
:10BAC8002021220071A300112DA400110000000004
:10BAD8000200000016BA00110000000059B1001160
:0CBAE800000000000200000014BA001171
:020000041FFFDC
:10000000000000001D3D001150B800114CB8001157
:100010009C5BFF1F000000000000000000000000CB
:1000200000000000000000000000000000000000D0
:1000300000000000000000000000000000000000C0
:1000400000000000000000000000000000000000B0
:1000500000000000000000000000000000000000A0
:100060000000000000000000000000000000000090
:100070000000000000000000000000000000000080
:100080000000000000000000000000000000000070
:100090000000000000000000000000000000000060
:1000A0000000000000000000000000000000000050
:1000B0000000000000000000000000000000000040
:1000C0000000000000000000000000000000000030
:1000D0000000000000000000000000000000000020
:1000E0000000000000000000000000000000000010
:1000F0000000000000000000000000000000000000
:1001000000000000000000000000000000000000EF
:1001100000000000000000000000000000000000DF
:1001200000000000000000000000000000000000CF
:1001300000000000000000000000000000000000BF
:1001400000000000000000000000000000000000AF
:10015000000000000000000000000000000000009F
:10016000000000000000000000000000000000008F
:10017000000000000000000000000000000000007F
:10018000000000000000000000000000000000006F
:100190006D2DFF1FCD2BFF1FC16601000000000069
:1001A000000000000000000000000000000000004F
:1001B000000000000000000000000000000000003F
:1001C000000000000000000000000000000000002F
:1001D000000000000000000000000000000000001F
:1001E000000000000000000000000000000000000F
:1001F00000000000000000000000000000000000FF
:1002000000000000000000000000000000000000EE
:1002100000000000000000000000000000000000DE
:1002200000000000000000000000000000000000CE
:1002300000000000000000000000000000000000BE
:1002400000000000000000000000000000000000AE
:10025000000000000000000000000000000000009E
:10026000000000000000000000000000000000008E
:10027000000000000000000000000000000000007E
:10028000000000000000000000000000000000006E
:10029000000000000000000000000000000000005E
:1002A000000000000000000000000000000000004E
:1002B000000000000000000000000000000000003E
:1002C000000000000000000000000000000000002E
:1002D000000000000000000000000000000000001E
:1002E000000000000000000000000000000000000E
:1002F00000000000000000000000000000000000FE
:1003000000000000000000000000000000000000ED
:1003100000000000000000000000000000000000DD
:1003200000000000000000000000000000000000CD
:1003300000000000000000000000000000000000BD
:1003400000000000000000000000000000000000AD
:10035000000000000000000000000000000000009D
:10036000000000000000000000000000000000008D
:10037000A5B1001100000000000000000000000016
:10038000000000000000000000000000000000006D
:10039000000000000000000000000000000000005D
:1003A000000000000000000000000000591AFF1FBC
:1003B000000000000000000000000000000000003D
:1003C000000000000000000000000000000000002D
:1003D000000000000000000000000000000000001D
:1003E000000000000000000000000000000000000D
:1003F00000000000000000000000000000000000FD
:081838007069FF1F4118FF1F3A
:10184000024981F3088801F0B7FF00007069FF1FAB
:1018500010B501F0E1FF072804D0122808D00228B3
:1018600008D010BD044A0420136B01331363F8E75A
:101870000220F6E71420F4E7585FFF1FF8B50700D1
:101880000C0026002500503630785135002804D150
:101890000300287058342370F8BD2978CA00481E08
:1018A0008141A3183800A25C5B68C9B2FFF7D0FF82
:1018B00000280DD12B78DA00A218013350602B706C
:1018C0003378044A013B3370136A01331362D8E75B
:1018D0000123DFE7585FFF1F5C234343074910B52F
:1018E000C9180B0058331B78012B05D1FFF7C6FF31
:1018F000034A936A0133936210BDC0468C5FFF1F99
:10190000585FFF1F10B501F0C7FE064A0121130002
:1019100010CB4942D967044B136002F0BDF8200098
:1019200010BDC04600E100E01000100010B504003A
:1019300001F0B2FE024B1C6002F0AEF810BDC046D2
:1019400000E100E0431E5A425341A022F0B5D2010B
:101950005B421340154D164A40019B182A18127E0F
:101960008BB00191002A1BD01A000832D46F0022DC
:10197000E6B206AFE4B294420EDC2818C369002B2D
:1019800008D0019902AA117106AA049202AA16733C
:1019900003A898470BB0F0BD1978B9540132EAE7B3
:1019A0001A7D1A7806AB01261A70E6E71862FF1F47
:1019B00000400040F0B5254B04004001C25C85B0FA
:1019C000002A2BD01A18117E002927D0917E0029D9
:1019D00024D01179022921D11689D788D168F51B25
:1019E000ADB22A1C102D00D9102292B2BE4217D1DE
:1019F0001818012303710023C269C38003819A422E
:101A000006D06846032103730171029301A8904731
:101A10000820002C00D0192001F08EF805B0F0BD90
:101A2000013C65426C41A0256442ED012C40084D0B
:101A30001B186419074D0633013A92B2AA42EDD041
:101A40001888461C1E80085C2070F5E71862FF1F8E
:101A500000400040FFFF00000F220E4B10B59868B9
:101A6000104002380A280BD801F0F0FD0D0A0B0ACD
:101A70000A110A0A0A0A060002210020FFF762FF83
:101A800010BD0121F9E70020FFF794FFF8E7DB6FB5
:101A9000F6E7C046004000400F220E4B10B5986894
:101AA000104002380A280BD801F0D0FD0E0A0B0AAC
:101AB0000A120A0A0A0A060002210120FFF742FF61
:101AC00010BD01210800F9E70120FFF773FFF7E7D8
:101AD000DB6FF5E700900040564B70B51B68012B9B
:101AE00003D1554A936D0133936501F015FF534BB4
:101AF000534A1860534B544C1A600123534A1360E5
:101B0000534A13602378002B06D0062251495248CD
:101B100001F042FE00232370504A514B10681B789D
:101B2000C1B2002B0ED14F4CC0B223785BB2002B58
:101B30004FDB237824785BB264B21B0424021B19A8
:101B40001B1813600B1C50294ED95023464A474995
:101B50001078DBB2FF2202284BD10868444C454D77
:101B6000267890432A78964254D9227824782E7881
:101B7000023B5D10A31B6B435201D31A10335B1160
:101B80001843086001F080FF031F012B45D83A4B32
:101B90001B78002B06D0394B1B78002B02D000207D
:101BA00001F022FFA122364B92009978354B4A432F
:101BB0001B689B18832292009B181B78033B012B08
:101BC00003D8AF20400001F08FFD01222E4BDA82B6
:101BD00070BD237824785BB264B2FF33FF341B04FA
:101BE00024021B190138ABE7CAB2022AAED2022383
:101BF000ACE70868254C264D267890432A78964213
:101C000008D9227824782D78023B5B10641B63434B
:101C10005201B2E72378DBB2B2E70228D5D11D4BDF
:101C20001B78013B022B03D91B4B1B78022BCCD119
:101C30006C20C8E79809FF1FFC0FFF1F905EFF1F75
:101C4000FF3F000014100340945EFF1F0C10034080
:101C500000100340D50BFF1F7211FF1FB40003409B
:101C60008C09FF1F680AFF1F490AFF1F94000340E9
:101C7000460AFF1F470AFF1FF908FF1F2209FF1F1F
:101C8000300DFF1F3409FF1FBC0BFF1F440AFF1F4D
:101C9000450AFF1F1C09FF1F2309FF1F10B501F094
:101CA0001BFE0022014B1A8010BDC0468C5EFF1F38
:101CB00070B5244D2B68002B28D001F025FE2B6831
:101CC000D8402B680400002B27D001F0A5FE2B681C
:101CD000D8401D4B1D4A9978A1239B004B431268A5
:101CE000D118D25C91239B00002A20D0CA5801321F
:101CF000CA50174B17491B680868834214D3D23B5C
:101D0000181A012A1AD0144B186070BD01F0FCFD9E
:101D1000124B196801F0C8FED3E701F07DFE0F4BAE
:101D2000196801F0C1FED4E70D495B18E8E7CA5015
:101D30000C4B1B68DB68E418201AE4E7F530FF3031
:101D4000E1E7C0461C08FF1F300DFF1F3409FF1FCD
:101D50009C09FF1F905EFF1FA009FF1F1808FF1FAF
:101D60002DFF3F00985EFF1F70B504000D0028296D
:101D700016D10300A433C2881B889B1A0B4A9BB25E
:101D800093420DD906006A3605223100653001F014
:101D90006BFE002804D13100200001F0DDFD70BD94
:101DA0002900200001F058FEF9E7C046FE7F000040
:101DB000F8B50500012001F0DFFC134CA36AA26A0C
:101DC0009342FBD1114E336001F08EFD10490300A8
:101DD00008601048426894460F4A17680022BC45C4
:101DE00001D24268BA1A0D4802603268AD18A422C6
:101DF000E562606A520302436262094A1278002A6D
:101E000001D00F3B0B60F8BD00F00040340AFF1F0B
:101E1000E408FF1F28100040180AFF1F1C0AFF1FBC
:101E20001C09FF1F70B580241025E405A3682B430F
:101E3000A36001F041FDA368AB43A36070BD000047
:101E4000F7B5160080221C001023D205019191687D
:101E500005000B43936000225A4BD7301A6001F003
:101E6000FBFC9D232A002F009B00EB58CA32012166
:101E70000092FC37002B01D00021009A386801F055
:101E8000DBFC2900009BCB311A784F4BD3351A600D
:101E90004B780A781B0213438A7812041A43CB78D2
:101EA0001B061343494A1BBA13604B790A791B027C
:101EB00013438A7912041A43CB7931001B0613436A
:101EC000434A1BBA13606B782A781B021343AA7823
:101ED00012041A43EB781B0613433E4A1BBA1360E5
:101EE000019A330213433C4A13603C4B22001B1BF4
:101EF0009C4603293DDCB3089A0013005142B21AF4
:101F0000032A46D1354AE018511A827840781204E3
:101F100000020243E05C043302430A600022FF2B0C
:101F20004BDDF0222E4B12011A600F222D4B1A604E
:101F30002D4A1368002BFCD00023224A2749136046
:101F4000091B321D0B191B68043A180A23706070B4
:101F5000180C1B0EA070E3700434002AF2DC8022FF
:101F600010213B68D20501333B6093688B4393603B
:101F7000F7BD6346D578981893782D061B042B433C
:101F8000157804392B43557804322D022B43036016
:101F9000AFE7022A0AD1114AE05C511AE2185278DE
:101FA000120202430A6004339BB2B7E7012AB5D19B
:101FB0000A4A521AE15C1160F5E7084959180A60AB
:101FC0000433ACE7000004403C0004403800044007
:101FD00034000440300004400C0004400001044080
:101FE000040004401000044014000440F7B515003C
:101FF00080221C001023D2050091916807000B433A
:1020000093600023654AD730136001F025FC9D23BF
:102010003E009B00F9583B00CA363200FC330029D1
:1020200000D07FE0586801F007FC390032785C4B43
:10203000CB311A604B780A781B0213438A78AC467E
:1020400012041A43CB78281D1B061343554A1BBAAA
:1020500013604B790A791B0213438A7912041A43DD
:10206000CB791B061343504A1BBA13604B7A0A7A8A
:102070001B0213438A7A12041A43CB7A21001B06EF
:1020800013434A4A1BBA1360009A2B021343484A6F
:1020900013602200474B1B1B0093009BCE785B18FC
:1020A00001938B7836061B0433430E780438334390
:1020B0004E78043136023343019E33600328ECDC52
:1020C0000321A808431C9B002940800003292BD131
:1020D0003849E5185E18A9786D78E35C09042D028B
:1020E000294319433160030008330021FF2B2DDD04
:1020F000314B324919600F21314B196001232749B7
:102100000B60304B19680029FCD006211B680B407E
:10211000042B20D080220020D20593680A318B4303
:102120009360FEBD01217DE7022908D121495D1898
:10213000E1184978E35C090219432960D3E70129D2
:10214000D3D11C495918E35C0B60CCE71948181827
:1021500001600433CAE7002310490B606346002B7B
:102160000CDC3B00FC335A68102101325A6080229B
:10217000D205936801208B439360D2E7009B9B18A4
:102180001B68190A13705170190C1B0ED3700423AD
:102190005B4291709C440432E0E7C046000004407A
:1021A0003C00044038000440340004403000044047
:1021B0000C0004400001044004000440080F00002B
:1021C000100004401400044010B5002901D001F0B3
:1021D000EBFA10BDF7B5604B01919978A1239B00F4
:1021E0004B435E4A060014681022E418D6235B00B5
:1021F000E0583623FF33E35C00279343222B41D181
:10220000574B0F3A1A600760012501F03DFA019B18
:102210001880E8235B00E35C002B01D0B34258DD5B
:102220000023504FFB70AD33FF33E3581A68002A88
:1022300003D09B88DB439B071DD03823FF33E35C2F
:10224000002B18D09B235B00E35C002B13D1D13310
:10225000FF33E35CB3420EDAA4235B00E15AE018DB
:10226000090A023101F0E8FB23000122FE33013E9E
:1022700001351A87FA70E8235B00E35C002B2AD053
:10228000A8B2FEBD03683D00002BBED0818804309B
:10229000090A023101F0D0FBD6235B00E3581F602E
:1022A000B2E72300B133BA00FF3398580137818871
:1022B0000430090A023101F0BFFBE8235B00E35C54
:1022C000BB42EEDCE822F61AED1800235200A354BC
:1022D000A6E70027F1E7200001F026FA00281FD02A
:1022E000002E1DDD7319882647190193B6002000C2
:1022F00001F06AFA5A308000201840680135818860
:102300000430090A023101F097FB200001F0FCF9CA
:10231000A3590133A351BD4202D0019B9D42E6D196
:10232000114BE35C002BABD095239B00E35C002BAF
:10233000A6D00E4BE15A0029A2D00D4AA35C9942C7
:1023400002D90133A3549BE700231A212000A35490
:1023500001F092F994E7C046300DFF1F3409FF1FCA
:1023600000140340E010FF1F5A0200007202000038
:102370005E0200000D4970B54A6E0D4CD2038B69A8
:10238000D20BA24206D80B4D0224AA4204D901F076
:1023900003FB70BD02246442E21815007E24254030
:1023A0002242F4D0A3432B438B61F0E700F00040BE
:1023B0000A200000FC1C00000B001B3B70B5040051
:1023C0003020E02B0DD81300E025493BFF3B9BB2AA
:1023D000ED00AB4205D8034B200019825A8201F070
:1023E0009BF970BD8410FF1FD722044B92009B58AD
:1023F00010B5002B00D0984710BDC0460000FF1F4D
:1024000010B501F0ADF8FFF7EFFF2749274BCA6D74
:10241000274C1A4084235B001343CB65254B1B6874
:10242000186A01F0A9F9244B244A1A60244B254A62
:102430001A60A022244B52001A60244B187801F035
:1024400083FA2000224901F08FF90023A3600233B0
:10245000A360204B2049236003232048A36001F0A0
:1024600083F910221E4BFF201A60802252031A604B
:10247000802292031A60802212041A6001F0B4FADA
:10248000012001F0D1FAFA20400001F07DFA582035
:1024900001F02AF9134801F0AFF9012001F01CF90D
:1024A000072001F011FB10BD00F0004000FEFEFF10
:1024B00014100040985EFF1F000003400180063D9D
:1024C000BC00034034080000A40003404A0AFF1F78
:1024D00071020000C3090000FFFF3F002810004008
:1024E00000E100E030750000674E336888331B68F8
:1024F00083F3088801F0E8F9644A6549136800200D
:102500000B401360634B644A1B68934200D1A6E002
:1025100001F0D2FA0221614A13688B431360FFF77E
:102520006FFF5F4B5F4C1878C0B201F055F9002384
:10253000A3600233A3605C4B0120236001F01CF90F
:102540000323A36001F0B8F8040001F0E5F90500E9
:1025500001F0B2F8554B186001F026FA544B196897
:10256000621A531EA14200D213008022D20393426A
:1025700001D39B029B0A3268D16AC90700D471E07B
:102580004C491C0C09689BB24C4359432402090A6C
:10259000641803264849FC3293680A6847489B1A26
:1025A000474A0768126847499B18474A9A183340B8
:1025B0009208DB190A600360042B03D9013233400F
:1025C0000A6003600E684149A619300001F06CFAF8
:1025D0003F4F3E493B68C3183B603000019301F018
:1025E00003F93C4E3068081838493060884205D9F4
:1025F000019B01333B6001F0F7F8316001F07CF999
:10260000354B1B78002B0DD001F086F9334B621B44
:10261000196812188A4232D24919091B091A30481E
:1026200001F0A2F82F4E337A002B0ED001F074F98E
:10263000621BF1681218914224D94919091B091A21
:10264000294801F091F800233372284B83F308885E
:1026500001F02AF8002001F02FFA01F08DF901F0C5
:102660002BFA5CE7DC0199000234641A5900641A01
:1026700009214B438033CB40A408E41889E7FA21B1
:102680008900CCE71A49DBE7985EFF1F1CF0004089
:10269000FFFFC1FF0C0AFF1FB641210310000040DD
:1026A000490AFF1F14100040C3090000100AFF1F51
:1026B000340AFF1F380AFF1F200AFF1F280AFF1FC6
:1026C0001C0AFF1F240AFF1FC4090000710200003A
:1026D0006008FF1F2C0AFF1F1C09FF1FE408FF1FD3
:1026E00000100040740BFF1F3C1000400000002051
:1026F000DC050000A022054B92009B5810B5002B72
:1027000001D0984710BD01F01FF8FBE70000FF1F44
:10271000A122054B92009B5810B5002B01D0984781
:1027200010BD01F011F8FBE70000FF1FA222054BCE
:1027300092009B5810B5002B01D0984710BD01F0B6
:1027400003F8FBE70000FF1FA322054B92009B58F4
:1027500010B5002B01D0984710BD00F0F5FFFBE746
:102760000000FF1FA422054B92009B5810B5002BC0
:1027700001D0984710BD00F0E7FFFBE70000FF1F06
:1027800070B501F0C9F84F4B186000F0D5FF040098
:10279000C30702D401F088F870BD00224A4B1A60CA
:1027A0004A4B18780138042829D800F04FFF03203D
:1027B000181C2400200001F057F80128ECD0444CEC
:1027C0002378042B6ED101F0CFF80028E4D001F07B
:1027D0002BF8582000F088FF02232370DCE720004C
:1027E00000F0BAFFE9E7200001F02EF8E5E720004D
:1027F00001F09AF8E1E7200000F0C6FFDDE701F004
:1028000043F90500012808D1324B1B78053B012B09
:1028100003D82000FFF76EFFD1E72D4B1B78022B6A
:1028200001D0052B20D1022D28D12B4B9B7BAB4314
:102830001CD12000FFF76CFF264B18780128BED171
:102840006405BCD4244925224B7B034205D1233A9D
:1028500013405A42534126331A000B7D9342AED99E
:10286000322001F0B9F8AAE7022D07D1194B1B78E5
:10287000052B11D12000FFF759FFDDE7012D0BD10A
:10288000012B03D12000FFF75FFF98E7062B03D150
:102890002000FFF767FF92E7200000F055FF022DB0
:1028A0008DD1C9E7032B04D10C4B987C01F044F87F
:1028B00072E7072B00D06FE7094B987B01F0A4F873
:1028C0006AE7C0469C09FF1F9809FF1F9009FF1F78
:1028D0002309FF1F1C09FF1FA60BFF1FBC0BFF1FB7
:1028E000D40BFF1F10B500F099FE10BDF7B50B0C0F
:1028F000FF270122009300233C001E001D00944688
:10290000019089B262469A4010000840184136187A
:10291000B6B2FF2F02D1012E00D19FB20098024023
:102920001A41AD18ADB2FF2C02D1012D00D19CB2DD
:102930000133102BE6D10320012E07D1012D04D144
:10294000019B2401E4191C700138FEBD102EFCD13E
:102950000238102DF9D00230F7E700008023F7B5D8
:102960009C46264B264F01932649274A274D284C43
:10297000284B02281AD1604638600868264E30403D
:10298000802636033043086001990978002909D16F
:102990001660224A2A60224A2260E0221968914386
:1029A000A03A1BE08021C9021160F2E766463E6052
:1029B0000F68194E3E408027FF023E430E6001998A
:1029C000097800290DD1176001280ED1154A2A6017
:1029D000154A2260E02219689143C03A0A431A60FE
:1029E000F7BD802189021160EEE7E0210F4A024322
:1029F0002A600F4A22601A688A43F0E74B0AFF1FD9
:102A0000E0000340D8000340900003400000034072
:102A10005000034040000340FFFFE3FF0280063DFB
:102A2000804508220180063D8066082200800698C5
:102A300080550822F8B51E4B80261A680020140025
:102A40003440324232D11A681A4F32431A6001229E
:102A50003B68063093433B6000F08EFE0122164D2A
:102A60002B681E432E603B680A2613433B60802779
:102A7000BF00124B1B683B4211D1013EF6B2FF2E44
:102A800009D17E220E4B1C682B68E40B1440934343
:102A900023432B6005E0082000F06EFEE9E7002EDE
:102AA000EFD180222B68600893432B60F8BDC046AD
:102AB000C4F000405CF0004018F0004068F00040B6
:102AC00060F0004010B500F0BFFF01215820034A1C
:102AD00000F0FAFDFFF7AEFF10BDC046600AFF1F11
:102AE00010B578220021034800F086FF00F064FF53
:102AF000002010BDA061FF1F70B5040000F0CCFDE8
:102B000000230C200B4A010059438D18515C002909
:102B10000DD0A14208D1012300246B7000F0ECFD20
:102B200000F0BAFF200070BD01330A2BEBD1122454
:102B3000F6E7C046A061FF1F70B5040000F0ACFDD1
:102B4000002319001D000D4A1078002806D0A0426D
:102B50000CD1557001310C320A29F5D1002B0AD164
:102B600000F02AFF00F098FF002070BD5078461E4C
:102B7000B0411B18EEE700F0BFFDF3E7A061FF1FB7
:102B8000F7B504000C20002384460E4D01926746E1
:102B90005F43E85D7E19A04212D000280BD10A4B9A
:102BA0009C4662461B7808331370019B70707C55FD
:102BB0007160B360FEBD01330A2BE8D10320F9E751
:102BC0000720F7E7A061FF1F9C61FF1F8020F8B579
:102BD000484BC0051B68C1248360474BFF251A681A
:102BE000012313434361454BA4001A68444B402121
:102BF0001A60444B1A68444B1A60444B1A59AA4352
:102C00001A51C52292009E58AE43314380269950F6
:102C10009F583F49F6010F403E439E509E588027E3
:102C20003602360A3043985080201A5900020A4072
:102C300002431A5104341A59364E3F04324080265A
:102C40003A431A511A5936061202120A32431A51DD
:102C500008341A5980260A4002431A51C3229200AE
:102C60009F58B446AF4337439F509F58294E0F405B
:102C700007439F509F5837408026360437438026AD
:102C80009F509F5836063F023F0A37439F50C0224D
:102C90001F59AF433A431A511A591202120A1643E6
:102CA000C6221E5192009C58AC4365462C439C5052
:102CB0009C5800250C4020439850C72080001A588B
:102CC000154C1140C02212020A431A50134B1B78B4
:102CD000DB08AB4201DC0020F8BD2378002B06D0D6
:102CE000A368002B00D0984701350C34EEE7122082
:102CF000F2E7C046C83DFF1FC43DFF1FB0F00040D3
:102D00009861FF1FB4F000409461FF1F00E100E0F4
:102D1000FF00FFFFFFFF00FFA061FF1F9C61FF1F7F
:102D2000030010B51F2809D80722002013400724EC
:102D300004490A78A24313430B7010BD00230620F8
:102D4000F5E7C0469C61FF1F054B06491B780A68E2
:102D500005485B0702401B0B134300200B607047C4
:102D60009C61FF1F1CF00040FFFFC1FF70B50C25E8
:102D7000FFF7EAFF0A4B1C780A4BE4086543ED189D
:102D8000002C01D1200070BD2B78002B06D06B6881
:102D9000002B00D09847013C0C3DF1E71220F2E7F0
:102DA0009C61FF1F9461FF1F1FB5002102220B00D1
:102DB00001910091052000F05FFD02230B490A6894
:102DC0001A42FCD120230393039B5A1E0392002B2B
:102DD000FAD1074A1368002BFCDA0B246C4420005C
:102DE000012100F011FD207804B010BD90C8004012
:102DF00000C8004013B504000A4B0193019B002B4F
:102E000001D1112016BDFFF7CFFF2300034004427C
:102E100005D0052000F0B0FC019B013BEDE7180058
:102E2000F0E7C046FFFFFF0707B500F035FC802242
:102E30000821D205936A0191002B01D107399162D3
:102E400002210C4A11600199481E01900029FAD113
:102E500003311160053101910199481E019000294B
:102E6000FAD11160002B02D18022D205936200F0CA
:102E700013FE07BD00C00040F0B52D4C89B023788B
:102E8000002B4FD1FEF73EFD02232A4F03903A68F4
:102E90001A42FCD120230693069B5A1E0692002B51
:102EA000FAD1254E3368002BFCDA0120FFF7A2FF90
:102EB000011E02D0112009B0F0BD030003220190D1
:102EC000009005AD9F2000F0D7FC0321280000F002
:102ED0009BFC02233A681A42FCD120230793079BEC
:102EE0005A1E0792002BFAD13368002BFCDA01201E
:102EF000FFF780FF0028DDD10398FEF717FDAA78C1
:102F00006B7811041B020B4329780B436360130099
:102F1000113B0A49052B07D801239340A3600B609E
:102F2000012323700020C6E780231B03F6E7C04679
:102F3000B03DFF1F90C8004000C800409808FF1F28
:102F40001E4B30B55A6818781D4B85B0D3185942BE
:102F50004B4101210093002300F096FC194B1A4AC3
:102F600002259A6300221A6510325A658022C42114
:102F70009D65164B1648D202DA6789004258154BF8
:102F800080241A4080231B041343435064234120B0
:102F90000393E40500F006FA402000F003FA6562AE
:102FA000039D6B1E0393002DFAD103236362FFF789
:102FB0003BFFA562FFF760FF05B030BDBC3DFF1FC2
:102FC00095FFFEF700C80040050001FF04E100E0A6
:102FD00000E100E0FFFF00FFF0B585B00700FEF75D
:102FE00091FC022305002D4C22681A42FCD12023BB
:102FF0000093009B5A1E0092002BFAD1284E336892
:10300000002BFCDA0120FFF7F5FE002803D0112485
:10301000200005B0F0BD234B2360022322681A4232
:10302000FCD120230193019B5A1E0192002BFAD15F
:103030003368002BFCDA0120FFF7DCFE0028E6D124
:10304000194B1F60022322681A42FCD120230293ED
:10305000029B5A1E0292002BFAD13368002BFCDA35
:103060000120FFF7C7FE0028D1D1104B23600223B7
:1030700022681A42FCD120230393039B5A1E039219
:10308000002BFAD13368002BFCDA0120FFF7B2FEE7
:10309000041EBCD12800FEF749FCB9E790C80040E7
:1030A00000C8004001000006A8C8004001800001DF
:1030B00010B50020FFF790FF10BD000010B5064BC3
:1030C00018705960FFF73CFF00211320034AFFF7F7
:1030D00057FD002010BDC046BC3DFF1F412FFF1F04
:1030E000F0B5040085B003920291FEF70BFC882234
:1030F00063035B0B52051A438023DB059D6A802323
:10310000274F0092BA68002601901B039A420CD9FF
:10311000F82326001B041E401C4206D08022214BAF
:1031200052025E6219680A431A60002D0BD100F04A
:10313000B3FA02221C4B1A608023DB055A62013A63
:103140009A6200F0A9FC0023039A934220D1002D3B
:103150000AD100F0A1FA144B03221D608023DB0585
:103160005A629D6200F098FC8023BA681B039A4261
:1031700008D9002E06D000220A4B0C495A621A6860
:103180000A401A600198FEF7D1FB002005B0F0BD9F
:10319000009A0299D2181278CA540133D4E7C04673
:1031A000B03DFF1F00C8004000C00040FFFFFEFF11
:1031B000F0B587B0029103920400FEF7A3FB0190E3
:1031C00000F06AFA802302250122234EDB053560D8
:1031D0005D629A6200F060FC204F3B682B42FCD19C
:1031E00020230493049B5A1E0492002BFAD11C4DF9
:1031F0002B68002BFCDA0120FFF7FCFD002802D031
:10320000112007B0F0BD2000039A029900F034FCB1
:10321000022304003A681A42FCD120230593059B3F
:103220005A1E0592002BFAD12B68002BFCDA0120E4
:10323000FFF7E0FD051EE3D100F02EFA8023032204
:10324000DB0535605A629D6200F026FC0198FEF7AE
:103250006DFBE0B2D5E7C04600C0004090C800401A
:1032600000C80040F0B5802489B00600FEF74AFB94
:10327000E405A36A02250393029000F00DFA0123EE
:10328000304F3D606562A36200F006FC2E4C23685F
:103290002B42FCD120230593059B5A1E0592002B3F
:1032A000FAD12A4D2B68002BFCDA0120FFF7A2FD92
:1032B000002803D01124200009B0F0BD244B236066
:1032C000022322681A42FCD120230693069B5A1E31
:1032D0000692002BFAD12B68002BFCDA0120FFF7B5
:1032E00089FD021EE6D11B4B03211E6003000190E5
:1032F0000090202000F0C0FA022322681A42FCD17C
:1033000020230793079B5A1E0792002BFAD12B68A4
:10331000002BFCDA0320FFF76DFD041ECAD100F07C
:10332000BBF980230322DB053C605A629C6200F0FB
:10333000B3FB039B002B01D1FFF776FD0298FEF74C
:10334000F5FAB8E700C0004090C8004000C800404F
:103350000100000694C8004007B500020191042254
:10336000000A01A9FFF724FF0EBD000073B5050098
:1033700005240B4AA3005B429B1819686B46DE1DAF
:103380003000FFF7B3FA022804D133782B55013C03
:10339000EFD276BD052CFCD00128FAD10230F8E737
:1033A000140900111F2807D8012380228340D20569
:1033B00091680B43936070473F2808D8012380220F
:1033C00020388340D20551690B435361F3E75F28EE
:1033D000F1D80123802240388340D205116A0B4383
:1033E0001362E8E71F2807D8012280218240C9051F
:1033F0008B6893438B6070473F2808D80122802157
:1034000020388240C9054B6993434B61F3E75F283D
:10341000F1D80122802140388240C9050B6A9343CC
:103420000B62E8E71F2810D880230200DB05153A5D
:103430001968012A06D820229143196019680A43A5
:103440001A60704701228240F6E73F2811D8802396
:103450000200DB05353AD968032A06D810229143C9
:10346000D960D9680A43DA60EBE70122203882404C
:10347000F5E75F28E5D842238022181A413B8340B4
:10348000D205516A99435162516A0B435362D8E79E
:1034900010B50400012813D1A022184992050B6829
:1034A0005B015B0913430B60154B164A1968114009
:1034B000154A0A431A60402219680A431A6010BD6F
:1034C0000028FCD101000A2000F0E6F921000B20C1
:1034D00000F0E2F9C0220A4B920019680A43402129
:1034E0001A601A688A431A60B022044912060B68EF
:1034F0005B015B0913430B60E1E7C04614F0004039
:103500001CF000407F00FEFF80FD010072B6074AFC
:103510001368013313600422054B1A600023054A27
:1035200013608022D2055360FEE7C0467808FF1F73
:10353000C0F00040C4F0004005490B68002B05D1E5
:10354000044A0A6004490A60044A13607047C0468E
:10355000140AFF1F841E0000380AFF1FC4F0004039
:103560000023034A1360034A1360034A1360704741
:1035700054F0004040F1004044F10040002310B5F9
:10358000184C8AB0009301932378012B27D0694609
:10359000012000F019FA002817D1009B124902936C
:1035A000019B06AA0393114B02A81B680493104BBE
:1035B0001B68059300F080F910220E4906A800F060
:1035C00053FA002804D1FF23237000200AB010BD55
:1035D0000123094A074902A8237000F06DF9012070
:1035E000F4E7C0469C5EFF1F102900110829001156
:1035F0000C29001120290011A05EFF1F13B5012422
:103600006946012000F0E0F9034B00940193FFF7B5
:10361000B5FF200016BDC046BB0B000010B5FFF77C
:103620009FFFFFF7EBFF002802D0024B984710BD29
:10363000FEE7C046E1A2000002B471464908490015
:10364000095649008E4402BC7047C04602B4714618
:1036500049084900095C49008E4402BC7047C046D5
:1036600003B47146490840004900095A49008E4494
:1036700003BC70470000000001B40248844601BC4E
:10368000604700BF53B9000001B40248844601BC42
:10369000604700BFCD0C010001B40248844601BC64
:1036A000604700BF75A9000001B40248844601BC10
:1036B000604700BF7997000001B40248844601BC0E
:1036C000604700BF156B010001B40248844601BC8D
:1036D000604700BF0167010001B40248844601BC95
:1036E000604700BFE512010001B40248844601BCF6
:1036F000604700BF7912010001B40248844601BC52
:10370000604700BF21A9000001B40248844601BC03
:10371000604700BF5976010001B40248844601BCED
:10372000604700BF116E000001B40248844601BC2E
:10373000604700BF71B0000001B40248844601BC7C
:10374000604700BFBD0B010001B40248844601BCC4
:10375000604700BFE917010001B40248844601BC7C
:10376000604700BF0934010001B40248844601BC2F
:10377000604700BF2D6C010001B40248844601BCC3
:10378000604700BF0189000001B40248844601BCC3
:10379000604700BFF935010001B40248844601BC0E
:1037A000604700BFE94C010001B40248844601BCF7
:1037B000604700BFE9D4000001B40248844601BC60
:1037C000604700BFADB1001101B40248844601BC9E
:1037D000604700BFD9B0000001B40248844601BC74
:1037E000604700BF8914010001B40248844601BC4F
:1037F000604700BF090E000001B40248844601BCC6
:10380000604700BF8D11010001B40248844601BC2D
:10381000604700BF3D71010001B40248844601BC0D
:10382000604700BFE927000001B40248844601BC9C
:10383000604700BF6DF6000001B40248844601BC39
:10384000604700BF2144000001B40248844601BC27
:10385000604700BF0534010001B40248844601BC42
:10386000604700BF8944000001B40248844601BC9F
:10387000604700BF0134010001B40248844601BC26
:10388000604700BF496D010001B40248844601BC95
:10389000604700BFC56D010001B40248844601BC09
:1038A000604700BF319E001101B40248844601BC4C
:1038B000604700BFDD0A010001B40248844601BC34
:1038C000604700BFDD3F000001B40248844601BCF0
:1038D000604700BFC9A9000001B40248844601BC8A
:1038E000604700BF8D82000001B40248844601BCDD
:1038F000604700BFBD5C010001B40248844601BCC2
:10390000604700BFD544010001B40248844601BCB1
:10391000604700BFE90B010001B40248844601BCC6
:10392000604700BFC95C010001B40248844601BC85
:10393000604700BFF535010001B40248844601BC70
:10394000604700BF4DF9000001B40248844601BC45
:10395000604700BFEDA5000001B40248844601BCE9
:10396000604700BF85C1000001B40248844601BC25
:10397000604700BF01D7000001B40248844601BC83
:10398000604700BF8552010001B40248844601BC73
:10399000604700BF8512010001B40248844601BCA3
:1039A000604700BFD1AE000001B40248844601BCAC
:1039B000604700BFC166010001B40248844601BCF3
:1039C000604700BFADAE000001B40248844601BCB0
:1039D000604700BFE1AC000001B40248844601BC6E
:1039E000604700BF6137010001B40248844601BC52
:1039F000604700BFED6B010001B40248844601BC82
:103A0000604700BFB70E000001B40248844601BC05
:103A1000604700BFC1F7000001B40248844601BC02
:103A2000604700BF6D0B010001B40248844601BC31
:103A3000604700BF6911010001B40248844601BC1F
:103A4000604700BFC115010001B40248844601BCB3
:103A5000604700BFED68010001B40248844601BC24
:103A6000604700BF51B8000001B40248844601BC61
:103A7000604700BFCD4C010001B40248844601BC40
:103A8000604700BF9573010001B40248844601BC41
:103A9000604700BFDD0C010001B40248844601BC50
:103AA000604700BF9DA9000001B40248844601BCE4
:103AB000604700BF090E000001B40248844601BC03
:103AC000604700BF016C010001B40248844601BC9C
:083AD000604700BFF90D010081
:103AD8000200000012BA00110100000040B80011F5
:103AE800020000000EBA001101000000183BFF1F81
:103AF8000200000048B80011010000001C5CFF1F14
:103B0800020000000CBA001103000000905BFF1FC8
:103B1800120000000200000012BA001101000000AB
:103B280088B80011020000000EBA00110100000060
:103B380085B800110200000092B8001103000000CF
:103B4800CB5BFF1F020000000CBA0011030000004D
:103B5800E05BFF1F020000000EBA00110100000028
:103B680084B800110200000090B8001103000000A2
:103B7800A15BFF1F020000000CBA00110300000047
:103B8800C25BFF1F0200000012BA00110100000012
:103B9800CCB80011020000000EBA001101000000AC
:103BA800613CFF1F02000000DEB8001101000000A8
:103BB800C3B80011020000000EBA00110100000095
:103BC800603CFF1F02000000DCB80011010000008B
:103BD800E85BFF1F020000000EBA001101000000A0
:103BE8005F3CFF1F02000000DAB80011010000006E
:103BF800B3B80011020000000EBA00110100000065
:103C08005E3CFF1F02000000D8B800110100000050
:103C1800AEB80011020000000EBA00110100000049
:103C28005D3CFF1F02000000D6B800110100000033
:103C3800A9B80011020000000EBA0011010000002E
:103C48005C3CFF1F02000000D4B800110100000016
:103C5800A4B80011020202020202000000000000E3
:103C680016150000F94A0011BD4A001120B90011CB
:103C780090011D0018001800FFFF0701020304054A
:103C8800060201060000000000000000000000001D
:103C9800000000000000000000000000000000001C
:103CA800030000000200000012BA00110100000029
:103CB80040B90011020000000EBA00110100000016
:103CC8001C3DFF1F020000004AB90011010000005E
:103CD800165CFF1F020000000CBA00110300000070
:103CE800805EFF1F020000000EBA001101000000F4
:103CF8001C3DFF1F0200000048B900110100000030
:103D0800185CFF1F020000000CBA0011030000003D
:103D1800785EFF1F12000000000100000000011182
:103D2800FFFF000050485936000000000000000066
:103D38000B000500F0000000B4000028002800284F
:103D48003075A000A000A000A00000080008E00155
:103D5800F0001000100010001000100010005000BB
:103D68005000500010001000D007000000000000B4
:103D78000F0001000500307507001000010081FFE9
:103D880000000000FF00000019700011216E0011F2
:103D9800B16B0011FFFF0100FF000000359A001110
:103DA800B1970011C9960011000000000000000042
:103DB80000000800040000003B0001085902E0016F
:103DC800882128000200000012BA0011010000003A
:103DD800D8BA0011020000000EBA0011010000005C
:103DE800493EFF1F020000000ABA0011010000004E
:103DF8005862FF1F020000000EBA00110100000007
:103E0800483EFF1F0200000008BA00110100000030
:103E1800463EFF1F020000000EBA0011010000001C
:103E2800443EFF1F0200000006BA00110100000016
:103E38003C3EFF1F180018001D00900102000003FF
:103E4800020200000200000012BA00110100000086
:103E5800ECBA0011020000000EBA001101000000C7
:103E68008C3EFF1F0200000004BA00110000000091
:103E780000000000020000000CBA0011030000005E
:063E88007862FF1F20FF1D
:040000051FFF184180
:00000001FF
